:10627C0001190000770101030200000301FA040078
:10628C00FA0500030A0A5A0B001E0C00FA0D000353
:10629C000E00040F0164100096120132130AFA1456
:1062AC00020215010117010A1801FA1905321A0127
:1062BC000A1B01FA1C05321FFFFF20FFFF23011EE2
:1062CC002400642A00FA2B00FA2C50782D003C2E66
:1062DC0000462F001E3000643250783300003432F8
:1062EC00FA350164360164370150380A643C0064A5
:1062FC003E003C3F000040FFFF411450420A5A430D
:10630C000AC84405324500B44600FA470106480263
:10631C00034C00FA4EFFFF500606510596520A3206
:10632C00530B46540A96560102570546580002591B
:10633C000A465A32FA5B010A5C0A325E000A5F00B6
:10634C00FE61FFFF64FFFF66000267FFFF6A0A3C05
:10635C006B00006C32967300007400007801327987
:10636C0001327EFFFF81FFFF84FFFF8500AF8600B7
:10637C00018700FA89010A8A00009900009D0A969B
:10638C009E00019FFFFFA0FFFFFAFAFA00007701C1
:10639C0001030200000301FA0400FA0500030A0AD3
:1063AC005A0B001E0C00FA0D00030E00040F0164C2
:1063BC00100096120132130AFA1402021501011789
:1063CC00010A1801FA1905321A010A1B01FA1C05F7
:1063DC00321FFFFF20FFFF23011E2400642A00FA56
:1063EC002B00FA2C50782D003C2E00462F001E302E
:1063FC0000643250783300003432FA3501643601CF
:10640C0064370150380A643C00643E003C3F000095
:10641C0040FFFF411450420A5A430AC84405324512
:10642C0000B44600FA4701034802024C00FA4EFF42
:10643C00FF500606510596520A32530B46540A96E3
:10644C00560101570546580001590A465A32FA5B63
:10645C00010A5C0A325E000A5F00FE61FFFF64FF06
:10646C00FF66000267FFFF6A0A3C6B00006C329605
:10647C007300007400007801327901327EFFFF81D5
:10648C00FFFF84FFFF85FFFF86FFFF87FFFF89016A
:10649C00028A00009900009D0A969E00019FFFFF52
:1064AC00A0FFFFFAFAFA0065006F00790083008DF7
:1064BC00009700A100AC00B600C000CA00D400DEFA
:1064CC0000E800F20058006000680070007800805E
:1064DC0000880090009800A000A800B000B800C18F
:1064EC0000C800D000D800DF00E600EE00F6004146
:1064FC000047004D00530059005F0065006C0071AF
:10650C000077007D00830089008F0095009B00A21E
:10651C0000A700AC00B200B900C000C500CA00D290
:0A652C0000D500DD00E100E700EFFC
:103A390090004AE0D3940440149007BCE0FEA3E050
:103A4900FF90627E12666FE493F59980129007BC2D
:103A5900E0FEA3E0FF90639812666FE493F59990F6
:103A690007BCE0FEA3E0FF90627CE493FC74019341
:103A7900FDEFB50507EEB50403754D009007BC12BF
:103A890066562275A71085F97385FA747E017F0041
:103A9900E574126648E5732FFF50010E8E5A8F5B4D
:103AA900900017E0FCA3E0FDEF2DFDEE3CFC8C5CE3
:103AB9008D5D2275A71085F97385FA747E017F00E3
:103AC900E574126648E5732FFF50010E8E5A8F5B1D
:103AD900AC2CAD2DEF2DFDEE3CFC8C5C8D5D22E513
:103AE9005DF5FBE55CF5FCD29322E55DF5E9E55C66
:103AF900F5EAD29422E55DF5EBE55CF5ECD291228D
:103B0900E55DF5EDE55CF5EED29222E55DF5FDE5C5
:103B19005CF5FED28722E55DF5CEE55CF5CFD29066
:103B290022AE5AAF5B74788E048F05FF1266388C0B
:103B39005C8D5DAE5AAF5B74788E048F05FF12669B
:103B4900638C5A8D5BE55B455A60137478C3955B4A
:103B5900FFE4955AFE8E5A8F5B785C12669CE5737A
:103B6900A85CB80015D3955D4010E573C3955DFF5A
:103B7900E4955CFE8E5C8F5D8010E5732403C3952C
:103B89005DFFE4955CFE8E5C8F5D2290008CE0B455
:103B99000104C2118002D21190008DE0B40104C267
:103BA900128002D2129000CAE075F0DCA4FFAEF0D8
:103BB900740A8E048F05FF1266389007B2ECF0A3E1
:103BC900EDF0A20D401674038C068D071266487439
:103BD900011200399007B0EEF0A3EFF07E017F00EB
:103BE900900088E01266489000CBE08E048F05FFB4
:103BF900126638740AFF1266388D609000D4E07539
:103C0900F0DCA4FFAEF0740A8E048F05FF1266384B
:103C19009007B6ECF0A3EDF09000D6E060139000A9
:103C2900D6E0F5F0741684FF7E00EF9007C4F080AB
:103C39000674649007C4F09000CCE090006FF09097
:103C49000116E0900059F09000A5E090005BF0901B
:103C590000CEE090005CF090007AE090005DF0907A
:103C69000100E0900062F0900164E0900063F09040
:103C79000165E0900064F0900166E0900065F0A2B3
:103C89002BB34016900164E0700C900165E070065A
:103C9900900166E060028002C22B74E390006EF02E
:103CA9009000B5E0B40B0874E390006EF0805A9070
:103CB90000B5E0B419129000CBE090649D12008C1D
:103CC900E49390006EF080419000B5E0B41E12902C
:103CD90000CBE09064BB12008CE49390006EF080FE
:103CE900289000B5E0B428129000CBE09064E5126A
:103CF900008CE49390006EF0800F9000B5E0B4461C
:103D0900089000ACE090006EF09000E5E0FE9000B5
:103D1900B3E06E600A9000B3E09000E5F0D22A901B
:103D29000072E0FE9000B2E0B50633900074E0FE48
:103D39009000D0E0B50627900073E0FE9000DEE029
:103D4900B5061B900076E0FE900085E0B5060F9061
:103D59000075E0FE9000C0E06E7003023F1890000D
:103D69004AE0C3940550087402900101F0801C9048
:103D790000C0E0640360069000DEE060087407900C
:103D89000101F08006740A900101F0900085E0B409
:103D9900010674009000EBF0900085E0B40206740F
:103DA900009000D0F0900085E0B403067400900004
:103DB900DDF09000B2E060147418900099F074007E
:103DC9009006C6F074009006C7F0800C740090004D
:103DD90099F074189006C6F09000D0E0D394014091
:103DE900147419900103F074009006CAF0740090DD
:103DF90006CBF0800C7400900103F074199006CA88
:103E0900F09000C0E0B403089000DEE064026002B4
:103E1900800674009000DEF09000DEE0B4010890A6
:103E290000C0E064036002801A741A900104F074FF
:103E39000090009AF074009006CEF074009006CFBE
:103E4900F080339000B2E0B4021A741A90009AF02C
:103E59007400900104F074009006CEF0740090068E
:103E6900CFF08012740090009AF07400900104F071
:103E7900741A9006CEF09000C0E0B402069000DEFD
:103E8900E06002801474049006DAF074059006DE8E
:103E9900F074069006E2F0802474009006DAF0745B
:103EA900009006DBF074009006DEF074009006DFE7
:103EB900F074009006E2F074009006E3F0D22A90C4
:103EC90000B2E0900072F09000DEE0900073F09094
:103ED90000D0E0900074F09000C0E0900075F09080
:103EE9000085E0900076F0900085E090005AF0900F
:103EF90000C0E090005EF09000DEE090005FF0907E
:103F090000B2E0900060F09000D0E0900061F09085
:103F190000E8E0B40117900023740FF0A374FFF0D8
:103F2900900025E4F0A3F074029000E8F09000E816
:103F3900E0B40341900025E0FEA3E0FF900023E0F8
:103F4900FCA3E0FD1266947410126648740812000E
:103F590039EF90006BF0EF700674FF90006BF0740E
:103F6900009000E8F0900024E090006CF0900023AD
:103F7900E090006DF0900079E090003DF090003DF8
:103F8900E00490003EF090003DE0240290003FF0F4
:103F990090003EE0D39403400B90003EE0C39403AD
:103FA90090003EF090003FE0D39403400B90003F17
:103FB900E0C3940390003FF07551019000BFE09079
:103FC9000040F0900040E0D39403400F900040E09F
:103FD900C39403900040F0D2248002C22490004090
:103FE900E004900041F0900040E02402900042F08B
:103FF900900041E0D39403400B900041E0C3940347
:10400900900041F0900042E0D39403400B900042AD
:10401900E0C39403900042F022C293C294C291C2B9
:1040290092C287C290E5B554EFF5B5E5B554DFF511
:10403900B5C296C295C2A0C297C2A2C2A1E5B554A3
:10404900BFF5B5E5B5547FF5B5E5B554FBF5B5C292
:1040590013755E469000C2E07005756D02800375A8
:104069006D0375550075540090000C74FFF0A3742E
:10407900DCF0C219C21BC21D74C8900037F074C8A5
:10408900900039F074C890003BF0755300755200E8
:10409900C20D754600E56FB40903756F00756300BD
:1040A900900019E4F0A3F0757010C216C217C21877
:1040B9009007B2E0FEA3E0FF740312664874011290
:1040C90000399007B0EEF0A3EFF0C2027557007502
:1040D9005600900010E4F0A3F0C22C7559007558F1
:1040E90000900084E075F032A4FDACF0900021EC62
:1040F900F0A3EDF0C23CA230B39205A231B392060F
:10410900A232B39207A233B39208A234B39209A29E
:1041190035B3920AA236B3920BA237B3920C227529
:10412900A71085F97385FA747E017F00E57412661C
:1041390048E5732FFF50010E8E5A8F5BAC5CAD5D65
:10414900EF2DFDEE3CFC8C5C8D5D123AE8123AF3E2
:10415900123AFE9000C0E0B40309123B09123B1465
:10416900123B1F75A7002285F97385FA747E017FBA
:1041790000E574126648E5732FFF50010E8E5A8FC1
:104189005B7E017F769000FDE0126648AC5AAD5B1C
:10419900ED2FFFEC3EFE8E5C8F5DE55DF5EDE55C98
:1041A900F5EE90006FE4F07412900046F02285F964
:1041B9007385FA747E017F00E574126648E5732FF2
:1041C900FF50010E8E5A8F5B9007B2E0FCA3E0FD11
:1041D900EF2DFDEE3CFC8C5C8D5DE55DF5FDE55C50
:1041E900F5FE22056422A2DBB340089000CCE090E2
:1041F900006FF0A2DCB34006C296C295C2A075D882
:10420900402285A77275A7109000C0E0640360077B
:104219009000DEE0B4022CA2D8B34002C293A2D926
:10422900B34002C294A2DAB34002C291A2DBB34006
:1042390002C292A2DCB34002C287A2DDB34002C22D
:1042490090802DA2D8B3400AC2939000DEE06002AC
:10425900C292A2D9B3400AC2949000DEE06002C2C1
:1042690087A2DAB3400AC2919000DEE06002C290F0
:1042790075D8408572A722900047E49364066002CE
:1042890080FE74C89007B8F8E4F0E8A3F075B500AB
:1042990075840175A70075FFA0900043E4F075C906
:1042A9001075A70F75A1C775A70075D90075CE0C34
:1042B90075A70F75F1FE75F2FF75F30775F478753B
:1042C900A4BA75A5FF75A60775AE0075AFFF75D4BD
:1042D9008175D5FF75D6FF75D7FF75A70075A20142
:1042E90075A14775F80975D80075D90475DD097583
:1042F900DE0975D84075A71075D80075D90475DA27
:104309000975DB0975DC0975DD0975DE0975DF09D4
:1043190075D84075A70075E60875E71075BC017575
:10432900BE0475BD6C75BE0775BDA075BE0875BDAB
:104339000175BC0075BB1875BC2075BA0875E88095
:1043490075D11375A70F75E10575E20075C74012A0
:104359004022759700759780740A1266287597C070
:10436900E5975420700280F8758F0275A700D2AFC7
:1043790075980075A90C75A70F75AB4375ADFB75DD
:10438900AC1E75A71075C91875CA0075CB0075C81C
:104399000475A700758912758E04758C00758A00DD
:1043A900C2A9D28C758D00758B00D2ABD28E75EFF8
:1043B9000675D944C29974C8F5097508001200E94F
:1043C90075B5001204E974639007B8F8E4F0E8A33E
:1043D900F012037574C89007B8F8E4F0E8A3F07414
:1043E90064F5097508001200E990005AE09000850B
:1043F900F0900085E0D39403400C7400900085F0A0
:10440900740090005AF0C221900085E0905E8DF80A
:104419002828738028A2B44002D221802075A70FD2
:1044290075F30F75A700A2A34002D221800F75A7CB
:0D4439000F75F31775A700A2A44002D22151
:0C5E8D0002441C02441E0244260244375A
:10444600A221B3405F757308E573D3940E5020E53F
:10445600739007B8F8E4F0E8A3F01202447464F528
:10446600097508001200E97873740126F650D974AC
:10447600029000C1F090005AE0900085F09000850F
:10448600E0905E99F8282873801674009000EBF08F
:10449600800E74009000D0F0800674009000DDF06D
:0C5E990002448E0244900244980244A08F
:1044A600D220805D757301E573D394075020E573C0
:1044B6009007B8F8E4F0E8A3F01202447464F50932
:1044C6007508001200E97873740126F650D9740154
:1044D6009000C1F090005AE0900085F0900085E0D1
:1044E600905EA5F8282873801674009000EBF08083
:0F44F6000E74009000D0F0800674009000DDF08E
:0C5EA5000244ED0244EF0244F70244FF07
:10450500C220900059E0900116F090005AE090000A
:1045150085F090005BE09000A5F090005CE09000D5
:10452500CEF090005DE090007AF090005EE09000A3
:10453500C0F090005FE09000DEF0900060E0900039
:10454500B2F0900061E09000D0F0900062E0900140
:1045550000F0900063E0900164F0900064E0900149
:1045650065F0900065E0900166F0900164E0700CE4
:10457500900165E07006900166E060028004C22B40
:104585008002D22B9000CBE07006740A9000CBF02D
:104595009000ACE0700674E39000ACF09000B2E0DF
:1045A50004900072F09000B3E09000E5F0123B94A7
:1045B500E5B54401F5B57406900048F07401900026
:1045C50049F0740390004BF0740590004CF0743181
:1045D50090004DF0740590004EF090004AE0B40450
:1045E50006740490004EF0740190004FF074009032
:1045F5000054F07400900057F074FF900058F07468
:104605004D90014FF07469900150F0747490015110
:10461500F07473900152F07475900153F0746290C8
:104625000154F07469900155F07473900156F0745B
:1046350068900157F07469900158F0742090015901
:10464500F0743690015AF0744390015BF0747990E0
:10465500015CF0746C90015DF09000E7E090006BF8
:10466500F090009EE090006CF090009FE090006D4F
:10467500F0A2B6B3920FA2B6B3920EA2B3B3921044
:10468500A2A4B39227A2B4B39228A2A3B39229906D
:104695000067E4F0756F00743A900778F074FD9048
:1046A5000779F0900068E4F09007B2E0FEA3E0FF20
:1046B500740312664874011200399007B0EEF0A336
:1046C500EFF0756E01900046E4F0C226756300C2F6
:1046D50014D215C202757100C22ED203C22FD204A4
:1046E500C230D205C231D206C232D207C233D20895
:1046F500C234D209C235D20AC236D20BC237D20C65
:10470500C222C223C224C225C22A12009E755F009E
:10471500756B0075610075653275660075670075A6
:104725006800756900756A00900019E4F0A3F075DA
:104735006C00D2B2D2A4D2B0D2B1D2A3D2A7D2A6A3
:10474500D2A5D2B7900084E0D394FA400674FA90CB
:104755000084F07E017F0090006DE01266489000B5
:104765006CE02FFF50010E900023EEF0A3EFF0EF69
:10477500D394FFEE940F4007900023E4F0A3F0904C
:10478500006BE0700674FF90006BF09000C1E0D301
:104795009402400674019000C1F09000C2E07005DB
:1047A500756D028003756D039000C3E0D3940140DD
:1047B5000674009000C3F09000C9E0C3940A500647
:1047C500740A9000C9F09000D3E07006740190005F
:1047D500D3F09000D3E0B4FF0674FE9000D3F090C0
:1047E50000DAE0D394FE400674FE9000DAF0900102
:1047F50000E0D3940240067401900100F090011688
:10480500E0D3940140067401900116F07401900004
:10481500E0F074019000E1F074009000E8F074009D
:10482500900108F074299006BEF0742A9006C2F033
:10483500741B9006D2F0741C9006D6F0D29C9000A2
:10484500B3E0D39404400674049000B3F0E570D34C
:10485500941040037570109006BFE0D3940C400689
:1048650074009006BFF09006C3E0D3940C40067424
:10487500009006C3F09006C7E0D3940C4006740080
:104885009006C7F09006CBE0D3940C4006740090D8
:1048950006CBF09006CFE0D3940C4006740090064A
:1048A500CFF09006D3E0D3940C400674009006D365
:1048B500F09006D7E0D3940C400674009006D7F02C
:1048C5009006DBE0D3940C400674009006DBF09074
:1048D50006DFE0D3940C400674009006DFF09006E6
:1048E500E3E0D3940C400674009006E3F0D2EC7537
:1048F500CF01A298B34005C298120646E54D600661
:10490500A299B3B340028005C299120C57E54E64D3
:10491500016005E54EB4040280D5C28E7E107F008D
:10492500E564126648E58D75F010A4FDACF0EF2D39
:10493500FDEE3CFCE58B75F01084FF7E00ED2FFF4E
:10494500EC3EFE8E548F55D28E9000A5E0605690B9
:10495500001B12665690001BE0FCA3E0FD90001DB5
:10496500E0FAA3E0FBEDB5033CECB50238B21FA2BB
:104975000DB34013A21FB34008E5B54404F5B58057
:1049850006E5B554FBF5B590001DE0FEA3E0FF90EC
:10499500001FE0FCA3E0FDEF2DFDEE3CFC90001DAB
:1049A500ECF0A3EDF09000B2E060099000B2E0C336
:1049B50094034002806F122D96A20DB3500990000A
:1049C50067E0C3940B4002800690009CE0F545E546
:1049D5004575F005A4FFAEF09007BAEEF0A3EFF031
:1049E500900089E0C395614007E55FC39560500776
:1049F5009007BAE4F0A3F0AE2EAF2F9007BAE0FC13
:104A0500A3E0FDEFD39DEE9C4004C297800B900080
:104A150067E0C394115002D2979000B2E0B402054A
:104A2500A297B392A19000B2E0B4031C122EB1AECE
:104A35002EAF2F9007BAE0FCA3E0FDEFD39DEE9CCF
:104A45004004D2978002C297A2B3301001B340410F
:104A5500A2B3301001B34039A2B3301201B3400CF8
:104A6500A2B6B34002D222A212B39210A212B33060
:104A7500B301B3401CA2129210A2B6B3300E01B31B
:104A85004004B20E800BA213B34006740590004695
:104A9500F0A2B6300F01B35003024FF3A2B6300FA8
:104AA50001B35003024FF3A2B6301101B350030214
:104AB5004E4F756E00A2B3B3B35006900077E06019
:104AC5000280067404900046F0900077E004F0A29E
:104AD500B3B34007900077E4F0800D900077E0B421
:104AE50003067404900046F0055EA2B3B3B3500606
:104AF500A213B3B34003024BB6E56DB4032EA22C4B
:104B0500B34022E55EB40403756D01E55EC394040C
:104B150050069000467401F0E55ED3940440067497
:104B250002900046F0755E01D22C805AE56DB40204
:104B350006756D01755E04E55EB40405755E01805C
:104B450045900046E07030E55EC394045006900041
:104B5500467401F0E55ED394044006740290004665
:104B6500F0E55EC394045002D226E55ED39404407A
:104B750002D226C296C2959000C2E0B40105124049
:104B8500228003755E01A222B34006A224922380EF
:104B950002B223C222A2B4B34002C228A2A4B340E7
:104BA50002C227A2A3B34002C229A226B34002C271
:104BB50026E55EB403549000A5E060099000A5E0E9
:104BC500C3943D4002804390001BE0FEA3E0FF90AC
:104BD50000A5E08E048F05FF12663874018C068DE2
:104BE5000712003990001FEEF0A3EFF090001FE0D0
:104BF500F8A3E090001DC8F0A3C8F090001BE4F0F6
:104C0500A3F0C21FE5B554FBF5B5AE58AF59AC548A
:104C1500AD55EF2DFDEE3CFC8C588D59AE54AF557E
:104C2500EFD39DEE9C4011900013E0FAA3E0FBEB5F
:104C3500C394E8EA94034002800690001312665676
:104C450090000CE554F0A3E555F090000EE554F006
:104C5500A3E555F0AE54AF55740C8E048F05FF12C5
:104C650066388C568D57C28E758D00758B007564B0
:104C750000755501755400D28E90000CE0FEA3E03E
:104C8500FFEF4E600B7CAC7D601265368E528F5304
:104C9500AE52AF537428BE00039F5010E5632FFF3B
:104CA50050010E74011200398E528F538553639053
:104CB50000C9E0A852B8000DD395534008E55390BC
:104CC5000045F080099000C9E014900045F0E56DBD
:104CD50060067553007552009000C0E0B40308905B
:104CE5000040E0655E6002800BA223B34004D2253C
:104CF5008002B225E55E64016005E55EB4030990B6
:104D050000B2E060031223D2E56FB40903756F00AA
:104D1500A214B35006A213B3B34003024DC89000CA
:104D25007EE0B40173900100E0B40214120E2690E7
:104D35000070E075F0BEA4FFAEF08E5C8F5D80560E
:104D4500E56775F00A84FF7E0090057812666FE0CE
:104D5500F55B755A00AE5AAF5B9000A3E01266484A
:104D650074648E048F05FF1266388C5C8D5DE55D7D
:104D7500900012F0AE5AAF5B90007CE0126648746A
:104D8500648E048F05FF12663874BE8C068D07127B
:104D950066488E5C8F5D801790007CE075F0BEA440
:104DA500FFAEF08E5C8F5D9000A3E0900012F0E501
:104DB50061C394CC5006E55D455C700280031241E9
:104DC50028D214E56DB40106A213B3B340028009DD
:104DD5007570019000477401F0E56D70689000C52D
:104DE500E0600D90006FE0A852B8000695534002B0
:104DF50080299000C5E0B40208757003756C0080C9
:104E05000CC200756C00900019E4F0A3F090006FDF
:104E1500E060067409900046F0802A7570019000E4
:104E25003DE0B55E069000477401F090003EE0B5A8
:104E35005E067402900047F090003FE0B55E067490
:104E450003900047F0A211B3920FA211B330B6013F
:104E5500B35003024FF3756E01E5B54401F5B57422
:104E65000B900067F0A211920FE55ED394484014B1
:104E7500D213E55ED3944E400B7405900046F0D2F4
:104E850026755E469000CDE0B40107E56AC394142B
:104E9500400280091240227413900046F0A22E3081
:104EA5000301B35017A22EB34008E5B54408F5B584
:104EB5008006E5B554F7F5B5A22E9203A22F30046E
:104EC50001B35017A22FB34008E5B54402F5B580EC
:104ED50006E5B554FDF5B5A22F9204A230300501C3
:104EE500B3500FA230B34004D2978002C297A230CC
:104EF5009205A231300601B3500FA231B34004D25E
:104F0500A28002C2A2A2319206A232300701B3509A
:104F15000FA232B34004D2A18002C2A1A2329207ED
:104F2500A233300801B35017A233B34008E5B544A6
:104F350040F5B58006E5B554BFF5B5A2339208A294
:104F450034300901B35017A234B34008E5B54480A5
:104F5500F5B58006E5B5547FF5B5A2349209A235BD
:104F6500300A01B3500FA235B34004D2928002C279
:104F750092A235920AA236300B01B3500FA236B376
:104F85004004D2878002C287A236920BA237300C2A
:104F950001B3500FA237B34004D2908002C290A251
:104FA50037920CE56AC394415009740E900046F09F
:104FB50012402290004EE0FE90004AE004C39E405D
:104FC5000990004AE0D39408400974FB900046F02C
:104FD500124022900053E06015900053E0FE9000CF
:104FE5004DE06E600974FE900046F0124022A22644
:104FF500B34006C296C295C2A09000FDE0600CAE1B
:1050050052AF537414BE00059F400280489000853E
:10501500E0905EB1F8282873803BA2B4B35005A296
:1050250028B340028005124170D2288028A2A3B37C
:105035005005A229B340028005124170D22980157E
:10504500A2A4B35005A227B340028005124170D235
:0550550027800280002D
:105EB10002501D02501F025032025045025058023A
:025EC100505A35
:10505A00A216B3B35008900040E0655E60030250A8
:10506A00EFA201B35006A200B3B3400280719000D0
:10507A00C0E0B40343123A8CA20DB34021A225B377
:10508A004005123AE88003123B099000DEE0B401C1
:10509A000BA202B34004D2A18002C2A18018123A24
:1050AA00E8123B099000DEE0B4010BA202B340040F
:1050BA00D2A18002C2A180249000DEE0C3940250F3
:1050CA000F123A8C123AE8A202B34002D292800C32
:1050DA00123A8C123AE8123ABC123B0975A700C27E
:1050EA0016D217D218A217B3B35008900041E06540
:1050FA005E6003025184A201B35006A200B3B3401A
:10510A000280719000C0E0B40343123A8CA20DB33E
:10511A004021A225B34005123AF38003123B1490B2
:10512A0000DEE0B4010BA202B34004D2A18002C2A5
:10513A00A18018123AF3123B149000DEE0B4010B7E
:10514A00A202B34004D2A18002C2A180249000DE50
:10515A00E0C39402500F123A8C123AF3A202B340FF
:10516A0002D287800C123A8C123AF3123ABC123BE2
:10517A001475A700D216C217D218A218B3B35008D2
:10518A00900042E0655E6003025219A201B3500624
:10519A00A200B3B3400280719000C0E0B40343128E
:1051AA003A8CA20DB34021A225B34005123AFE80E3
:1051BA0003123B1F9000DEE0B4010BA202B34004CD
:1051CA00D2A18002C2A18018123AFE123B1F90009F
:1051DA00DEE0B4010BA202B34004D2A18002C2A154
:1051EA0080249000DEE0C39402500F123A8C123AE7
:1051FA00FEA202B34002D290800C123A8C123AFEFE
:10520A00123ABC123B1F75A700D216D217C218E574
:0F521A0070905EC3F828287302565A9000B3E0D4
:065EC300025222025225EA
:10522900905EF6F8282873121EAE8012121EAE8008
:0E5239000D121F388008121FE48003121FE4BC
:0F5EF60002523002523502523A02523F025244D7
:1052470075700202565A122110122227A23CB3404F
:105257000C9000A7E0F56C7410900046F090007871
:10526700E0256CF5369007B0E0FEA3E0FF7414125A
:10527700664890000EE0FCA3E0FD74068F02FF1263
:1052870066388D078C038E048A058B061265369067
:1052970007B4EEF0A3EFF09000CEE0B40108744637
:1052A700BE00059F4002800D74469007B4F8E4F0F5
:1052B700E8A3F0801B9007B4E0FEA3E0FF74F0BE04
:1052C70000039F500B74F09007B4F8E4F0E8A3F0E4
:1052D700E53670037536019007B4E0FEA3E0FFE5FD
:1052E700362FFF50010E9007B4EEF0A3EFF0757064
:0552F70003900047E0F8
:035EC90002524D35
:1052FC00905F05F82828738019A23D400375700A49
:10530C008010A23D400375700B8007A23D400375D1
:02531C00700C13
:0C5F050002530302530502530E0253170F
:10531E0002565A9006BFE060031224EA9000FEE0A7
:10532E00B401149000FFE0A852B800049553500742
:10533E00E55FC39560400280097415900046F00247
:10534E0053D19000B3E0D39402403F900087E02405
:10535E0003A852B8000495535009900089E0D395E4
:10536E006150028008D2017408900046F0900087C8
:10537E00E0A852B80005D39553500B900089E02455
:10538E0003C395615002C2018039900087E0240367
:10539E00A852B8000495535007E55FC395604002CC
:1053AE008008D2017408900046F0900087E0A85261
:1053BE00B80005D395535009E560240FC3955F508F
:1053CE0002C2019000CDE07007E56AC3941440025A
:1053DE008002D201A2014005757004800A7570101A
:1053EE00900019E4F0A3F0A20DB34029E56775F023
:1053FE000A84FF7E0090057812666FE0C3946950B0
:10540E0005122407800F9007B2E0F8A3E09007B0D2
:0C541E00C8F0A3C8F002565A9000B3E09A
:065ECC00025321025426DE
:10542A00905F11F8282873120F108012120F108043
:0E543A000D1210BE8008121170800312117046
:0F5F110002543102543602543B025440025445AC
:105448009006C3E060031225C675700502565A120D
:1054580012B07570069006C7E060031226B6900673
:10546800CBE0600312279202565A900012E06006C1
:10547800A20DB3B34002801D900012E02529FFAEB3
:105488002850010E8E288F29E55ED394015006908E
:105498000012E014F01214F67570079006CFE06061
:1054A8000312286E9006D3E0600312294A02565A66
:1054B800900100E0B40203120E9E1218F5757008F0
:1054C8009006D7E06003122A269006DBE0600312FC
:1054D8002B0202565A121CB1A216B35005A217B3DA
:1054E80040028006D216D217D2187570109006DFC7
:1054F800E06003122BDE9006E3E06003122CBA0290
:10550800565A02565A900038E0C394465008C2963C
:105518007446900038F085365B755A0090003DE07F
:10552800F573123B2AE55D900038F0900006E55AC5
:10553800F0A3E55BF0C21A9007B4E0F55AA3E0F5D2
:105548005B90003DE0F573123B2AE55D900037F073
:10555800900000E55AF0A3E55BF0C219E56DB401CF
:105568000575700B800375700302565A90003AE077
:10557800C3944650139000CEE0B40104C296800252
:10558800C295744690003AF085365B755A009000D3
:105598003EE0F573123B2AE55D90003AF090000872
:1055A800E55AF0A3E55BF0C21C9007B4E0F55AA3F6
:1055B800E0F55B90003EE0F573123B2AE55D900054
:1055C80039F0900002E55AF0A3E55BF0C21BE56DE7
:1055D800B4010575700C8003757003807590003CEC
:1055E800E0C3944650139000CEE0B40104C2968004
:1055F80002C2A0744690003CF085365B755A009054
:10560800003FE0F573123B2AE55D90003CF0900006
:105618000AE55AF0A3E55BF0C21E9007B4E0F55A1C
:10562800A3E0F55B90003FE0F573123B2AE55D903F
:10563800003BF0900004E55AF0A3E55BF0C21DE5DD
:105648006DB40103756D00757003800680048002D7
:025658008000D0
:105ED2000254570254720254B80254DD02550A02A7
:105EE200550D0255740255E5025654025656025695
:045EF2005802565AA2
:10565A00900037E0B55E0280030256F5A219406B4E
:10566A00900000E0FEA3E0FFEF4E605DAC52AD5348
:10567A00740ABC0033D39D402FAA56AB5774058ACF
:10568A00048B05FF1266388D068C07900000E0FC3B
:10569A00A3E0FDCFCECF12000374011200399000AF
:1056AA0000EEF0A3EFF08021AE56AF57900000E075
:1056BA00FCA3E0FD120003740A8E048F05FF126634
:1056CA0038900000ECF0A3EDF0D219AE54AF55902B
:1056DA000000E0FCA3E0FDEFC39DEE9C400D1241EB
:1056EA00B7D296C21974C8900037F0A219B3B35052
:1056FA0007900037E0B55E02800D1241B7D296746A
:10570A00C8900037F0C219900038E0B55E028003F5
:10571A000257A9A21A406B900006E0FEA3E0FFEF31
:10572A004E605DAC52AD53740ABC0033D39D402F1A
:10573A00AA56AB5774058A048B05FF1266388D0684
:10574A008C07900006E0FCA3E0FDCFCECF12000349
:10575A007401120039900006EEF0A3EFF08021AE3A
:10576A0056AF57900006E0FCA3E0FD120003740A4E
:10577A008E048F05FF126638900006ECF0A3EDF058
:10578A00D21AAE54AF55900006E0FCA3E0FDEFC379
:10579A009DEE9C400AC2967446900038F0C21AA246
:1057AA001AB3B35007900038E0B55E02800AC29679
:1057BA007446900038F0C21A900039E0B55E028053
:1057CA0003025868A21B406B900002E0FEA3E0FFB0
:1057DA00EF4E605DAC52AD53740ABC0033D39D40AA
:1057EA002FAA56AB5774058A048B05FF1266388DAB
:1057FA00068C07900002E0FCA3E0FDCFCECF12009A
:10580A00037401120039900002EEF0A3EFF0802138
:10581A00AE56AF57900002E0FCA3E0FD12000374FD
:10582A000A8E048F05FF126638900002ECF0A3ED91
:10583A00F0D21BAE54AF55900002E0FCA3E0FDEF9E
:10584A00C39DEE9C40181241B79000CEE0B401040B
:10585A00D2968002D295C21B74C8900039F0A21B5E
:10586A00B3B35007900039E0B55E0280181241B711
:10587A009000CEE0B40104D2968002D29574C8900A
:10588A000039F0C21B90003AE0B55E02800302596B
:10589A0032A21C406B900008E0FEA3E0FFEF4E60CE
:1058AA005DAC52AD53740ABC0033D39D402FAA5647
:1058BA00AB5774058A048B05FF1266388D068C0770
:1058CA00900008E0FCA3E0FDCFCECF1200037401E4
:1058DA00120039900008EEF0A3EFF08021AE56AF27
:1058EA0057900008E0FCA3E0FD120003740A8E043E
:1058FA008F05FF126638900008ECF0A3EDF0D21C79
:10590A00AE54AF55900008E0FCA3E0FDEFC39DEE56
:10591A009C40159000CEE0B40104C2968002C29564
:10592A00744690003AF0C21CA21CB3B35007900010
:10593A003AE0B55E0280159000CEE0B40104C2964A
:10594A008002C295744690003AF0C21C90003BE077
:10595A00B55E0280030259FCA21D406B900004E070
:10596A00FEA3E0FFEF4E605DAC52AD53740ABC007B
:10597A0033D39D402FAA56AB5774058A048B05FF73
:10598A001266388D068C07900004E0FCA3E0FDCF78
:10599A00CECF1200037401120039900004EEF0A376
:1059AA00EFF08021AE56AF57900004E0FCA3E0FD73
:1059BA00120003740A8E048F05FF126638900004E1
:1059CA00ECF0A3EDF0D21DAE54AF55900004E0FC0C
:1059DA00A3E0FDEFC39DEE9C40181241B79000CEA4
:1059EA00E0B40104D2968002D2A0C21D74C890000D
:1059FA003BF0A21DB3B3500790003BE0B55E0280B6
:105A0A00181241B79000CEE0B40104D2968002D2B7
:105A1A00A074C890003BF0C21D90003CE0B55E0245
:105A2A008003025AC6A21E406B90000AE0FEA3E061
:105A3A00FFEF4E605DAC52AD53740ABC0033D39D88
:105A4A00402FAA56AB5774058A048B05FF12663895
:105A5A008D068C0790000AE0FCA3E0FDCFCECF12A2
:105A6A000003740112003990000AEEF0A3EFF080EF
:105A7A0021AE56AF5790000AE0FCA3E0FD120003E6
:105A8A00740A8E048F05FF12663890000AECF0A3A0
:105A9A00EDF0D21EAE54AF5590000AE0FCA3E0FD33
:105AAA00EFC39DEE9C40159000CEE0B40104C2966F
:105ABA008002C2A0744690003CF0C21EA21EB3B37C
:105ACA00500790003CE0B55E0280159000CEE0B42D
:105ADA000104C2968002C2A0744690003CF0C21E25
:105AEA009000D0E0B402028003025C06900069E0F4
:105AFA00D395665064900069E0F4042566FE900030
:105B0A00D3E08E00F5F0E884FF7E008F73EFC39434
:105B1A0010500CEF8573F0A4FDACF08D7380037503
:105B2A0073FF900069E0D39573400B900069E0C35E
:105B3A009573F57180037571009000EEE0D395714D
:105B4A0040069000EEE0F5719000EFE0C3957150C9
:105B5A00069000EFE0F5718071900069E0C39566E8
:105B6A00FE9000D3E08E00F5F0E884FF7E008F738C
:105B7A00EFC39410500CEF8573F0A4FDACF08D7355
:105B8A0080037573FF85735B755A00900069E02581
:105B9A005BFFAE5A50010E8E5A8F5B74FFBE00092E
:105BAA00D39F4005855B7180037571FF9000EEE01D
:105BBA00D3957140069000EEE0F5719000EFE0C3D6
:105BCA00957150069000EFE0F571A20DB3B3500D38
:105BDA0090006AE0FE9000DBE0D39E5002800A74D7
:105BEA0007900046F0C2A2801375A710E5CDC395B1
:105BFA00714004C2A28002D2A275A700E56FC394C5
:105C0A0009500AA2EDB34005C2ED123050AE54AFAE
:105C1A00557450C39F74C39E400C900068E0C394AF
:105C2A005A4003025E8AA213B34009124022740644
:105C3A00900046F0A221B34008E5B54404F5B580CA
:105C4A0006E5B554FBF5B5A215B3500EE561D3943C
:105C5A00334007E561C394CC40028041900100E0E3
:105C6A00B40214120E26900070E075F050A4FFAE34
:105C7A00F08E5C8F5D800F90007CE075F050A4FF81
:105C8A00AEF08E5C8F5DE55D455C6011E5B5440163
:105C9A00F5B5740B900067F0124128D21590006890
:105CAA00E0D394014007E561C3941A40028002C21E
:105CBA00159006BFE060031224EAA22E300301B356
:105CCA005017A22EB34008E5B54408F5B58006E59D
:105CDA00B554F7F5B5A22E92039006C3E0600312FD
:105CEA0025C6A22F300401B35017A22FB34008E5EE
:105CFA00B54402F5B58006E5B554FDF5B5A22F9277
:105D0A00049006C7E060031226B6A230300501B33C
:105D1A00500FA230B34004D2978002C297A23092A9
:105D2A00059006CBE06003122792A231300601B338
:105D3A00500FA231B34004D2A28002C2A2A2319271
:105D4A00069006CFE0600312286EA232300701B334
:105D5A00500FA232B34004D2A18002C2A1A2329251
:105D6A00079006D3E0600312294AA233300801B330
:105D7A005017A233B34008E5B54440F5B58006E5AF
:105D8A00B554BFF5B5A23392089006D7E060031266
:105D9A002A26A234300901B35017A234B34008E5C9
:105DAA00B54480F5B58006E5B5547FF5B5A23492C1
:105DBA00099006DBE06003122B02A235300A01B318
:105DCA00500FA235B34004D2928002C292A23592F9
:105DDA000A9006DFE06003122BDEA236300B01B315
:105DEA00500FA236B34004D2878002C287A23692ED
:105DFA000B9006E3E06003122CBAA237300C01B311
:105E0A00500FA237B34004D2908002C290A23792B8
:105E1A000C900068E0C3945A5010E56FB4090990D9
:105E2A000068E004F0756F00803BE56FB409037504
:105E3A006F00755500755400758D00758B0075647B
:105E4A0000900067E0C394115008900067E004F0E6
:105E5A0080067411900067F0900067E0B41106E5BF
:105E6A00B554FEF5B5900068E0D394014007E56AA1
:105E7A00C3944140028009740E900046F0124022F9
:035E8A000248F4D7
:105F20000000010001400160018001A001C001E00A
:105F300002000300039603B603D603F40400050031
:105F40000512052405360548055A056C057E0590A1
:105F500005A805C005DE0600061406280646066EDE
:105F600006AE05CF00FF013F015F017F019F01BF2A
:105F700001DF01FF02FF039503B503D503F303FF20
:105F800004FF05110523053505470559056B057DFA
:105F9000058F05A705BF05CE05F1061306270645A3
:105FA000066D06AD06ED05DD0FAA0FA50F9F0F9A32
:105FB0000F940F8D0F870F800F780F710F680F6090
:105FC0000F570F4E0F450F3B0F300F250F1A0F0EB7
:105FD0000F020EF50EE80EDB0ECC0EBE0EAE0E9FBF
:105FE0000E8E0E7D0E6C0E5A0E470E340E200E0CC9
:105FF0000DF70DE20DCB0DB50D9D0D850D6D0D54FD
:106000000D3A0D200D050CE90CCE0CB10C940C765C
:106010000C580C3A0C1B0BFB0BDB0BBB0B9A0B79D4
:106020000B570B350B130AF10ACE0AAB0A870A6429
:106030000A400A1C09F809D409B0098C0967094308
:10604000091F08FB08D608B2088E086A084608230C
:1060500007FF07DC07B9079607730751072F070DDE
:1060600006EC06CA06AA068906690649062A060A31
:1060700005EC05CD05B0059205750558053C0520D4
:10608000050504EA04CF04B5049C048204690451A4
:1060900004390422040B03F403DE03C803B2039D96
:1060A000038903750361034D033B032803160304AF
:1060B00002F202E102D102C002B002A00291028209
:1060C0000273026502570249023C022F02220216A5
:1060D000020901FD01F201E601DB01D001C601BBAD
:1060E00001B101A7019D0194018B01820179017029
:1060F0000168016001580150014801410139013234
:10610000012B0125011E01180111010B010500FFE2
:1061100000FA0FA60FA00F990F920F8B0F840F7C20
:106120000F740F6B0F620F580F4E0F430F380F2C69
:106130000F1F0F120F050EF70EE80ED80EC80EB780
:106140000EA50E930E800E6C0E580E420E2C0E15E0
:106150000DFD0DE40DCB0DB10D950D790D5D0D3FD0
:106160000D200D010CE10CC00C9E0C7C0C590C3563
:106170000C100BEA0BC40B9E0B760B4F0B260AFD83
:106180000AD40AAA0A800A550A2A09FF09D409A8CA
:10619000097C0950092508F908CD08A10875084AA5
:1061A000081E07F307C8079D07730749072006F76E
:1061B00006CE06A6067E06570630060A05E405BF8B
:1061C000059B057705540532051004EF04CE04AE97
:1061D000048F047104530435041903FD03E203C75B
:1061E00003AD0394037B0363034B0334031E0308D3
:1061F00002F302DE02CA02B602A30291027F026D1E
:10620000025C024C023C022C021D020E020001F252
:1062100001E401D701CA01BE01B101A6019A018FB3
:106220000185017A01700166015D0153014A014156
:10623000013901310129012101190112010B010468
:1062400000FD00F700F000EA00E400DE00D900D312
:1062500000CE00C900C400BF00BA00B500B100AD57
:1062600000A800A400A0009C009900950091008E59
:0C627000008A008700840081007E007B13
:10009E007547009007BCE4F0A3F075310075300091
:1000AE00754D00754E00C239D23A74FE9007BEF8F7
:1000BE00E4F0E8A3F074FE9007C0F8E4F0E8A3F0D3
:1000CE0074FE9007CAF0745A9007CBF0745A9007DA
:1000DE00CCF0D23BC22DC23DC23822750B00750A40
:1000EE0000AE0AAF0BAC08AD09EDC39FEC9E4016F7
:1000FE0074FF12662875CF01780B740126F6500432
:10010E0018E436F650DB22900043E0B4AA1C9007A8
:10011E0078E0B43C159007B8E0FEA3E0FFEF4E6028
:10012E0009741EBE0004D39F5003020243755D0086
:10013E00755C0075F8099007B8E0FEA3E0FF740740
:10014E006F4E6006740E6F4E7006743A900778F01C
:10015E009007B8E0FEA3E0FF7408BE001ED39F40D8
:10016E001A7E017F089007B8E0FCA3E0FD1DBDFFDD
:10017E00011C1200038E5A8F5B801F9007B8E0FEA1
:10018E00A3E0FF740812668C8F048E057E017F0833
:10019E00CDCCCD1200038E5A8F5BAE5CAF5D740C6E
:1001AE00D39F74019E500302023EA2F9B3407EE536
:1001BE005D455C700375A382AE5CAF5D74016F4EDE
:1001CE00700375A300AE5CAF5D74026F4E700D9040
:1001DE0007B9E075F002A4FDACF08DA3AE5CAF5D87
:1001EE0074036F4E700375A300AE5CAF5D7403BEF7
:1001FE0000039F5013AC5AAD5BED2FFFEC3EFE900B
:10020E00007412666FE0F5A3AE5CAF5DEFB40B0940
:10021E00EEB401057414126628AE5CAF5DEFB40B3C
:10022E0007EEB4010375F80D785C12669C0201A806
:10023E00900043E4F022755D00755C0075F809903E
:10024E0007B8E0FEA3E0FF7408BE001ED39F401A5D
:10025E007E017F089007B8E0FCA3E0FD1DBDFF0105
:10026E001C1200038E5A8F5B801F9007B8E0FEA30E
:10027E00E0FF740812668C8F048E057E017F08CD18
:10028E00CCCD1200038E5A8F5BAE5CAF5D7411D372
:10029E009F74019E5003020374A2F9B3500302032C
:1002AE0071E55D455C700375A3D2AE5CAF5D740104
:1002BE006F4E700375A300AE5CAF5D74026F4E702F
:1002CE000D9007B9E075F002A4FDACF08DA3AE5C05
:1002DE00AF5D74036F4E700375A300AE5CAF5D74BB
:1002EE00046F4E700375A300AE5CAF5D74056F4E68
:1002FE00700375A300AE5CAF5D74066F4E70037530
:10030E00A300AE5CAF5D74076F4E700375A300AEB5
:10031E005CAF5D74086F4E700375A300AE5CAF5D8D
:10032E007408BE00039F5016AC5AAD5BED2FFFEC68
:10033E003EFE90006F12666FE5A3F075A300AE5CF3
:10034E00AF5DEFB41009EEB401057414126628AE59
:10035E005CAF5DEFB41007EEB4010375F80D785C79
:10036E0012669C02029722755D00755C0075F80995
:10037E00AE5CAF5D7417BE0004D39F500302044DF4
:10038E00A2F9B3500302044AE55D455C700375A300
:10039E00D2AE5CAF5D74016F4E700375A300AE5CA0
:1003AE00AF5D74026F4E700D9007B9E075F002A448
:1003BE00FDACF08DA3AE5CAF5D74036F4E70037534
:1003CE00A300AE5CAF5D74046F4E700375A300AEF8
:1003DE005CAF5D74056F4E700375A300AE5CAF5DD0
:1003EE0074066F4E700375A300AE5CAF5D74076F3D
:1003FE004E700375A300AE5CAF5D74086F4E700354
:10040E0075A300AE5CAF5D7408BE00039F500C90E8
:10041E00005012666FE5A3F075A300AE5CAF5D747D
:10042E00166F4E70057414126628AE5CAF5D7416AE
:10043E006F4E700375F80D785C12669C02037E2277
:10044E00900043E0B4AB0280030204E8755D0075D2
:10045E005C0075F809AE5CAF5D7412BE007CD39F74
:10046E004078A2F9B34070E55D455C700375A382D8
:10047E00AE5CAF5D74016F4E700375A300AE5CAFE2
:10048E005D74026F4E700D9007B9E075F002A4FD19
:10049E00ACF08DA3AE5CAF5D74036F4E700375A3AD
:1004AE0000AE5CAF5D7403BE00039F500990005513
:1004BE0012666FE0F5A3AE5CAF5D74116F4E700502
:1004CE007414126628AE5CAF5D74116F4E700375B6
:1004DE00F80D785C12669C020463229007C7E4F064
:1004EE0074649007B8F8E4F0E8A3F012037574C8CA
:1004FE009007B8F8E4F0E8A3F074FF900050F074A1
:10050E00FF900051F074FF900052F0740090004A7A
:10051E00F074FF900053F07400900055F074019049
:10052E000056F090005CE0B4371A900059E090004D
:10053E0050F090005AE0900051F090005BE0900077
:10054E0052F080469007C77401F074659007B8F8B2
:10055E00E4F0E8A3F012037574C89007B8F8E4F05D
:10056E00E8A3F090005CE0B4371A900059E09000D8
:10057E0050F090005AE0900051F090005BE0900037
:10058E0052F0800674029007C7F09007C8E4F0742A
:10059E00669007B8F8E4F0E8A3F012037574C890FB
:1005AE0007B8F8E4F0E8A3F090005BE0B4371290DF
:1005BE000059E090004AF090005AE0900053F0800D
:1005CE00769007C87401F074679007B8F8E4F0E805
:1005DE00A3F012037574C89007B8F8E4F0E8A3F01E
:1005EE0090005BE0B43712900059E090004AF09012
:1005FE00005AE0900053F0803E74029007C8F074E9
:10060E00689007B8F8E4F0E8A3F012037574C89088
:10061E0007B8F8E4F0E8A3F090005BE0B43712906E
:10062E000059E090004AF090005AE0900053F0809C
:10063E000674039007C8F022E54E64046006E5993F
:10064E0064FF60028031A2394004D2398027E54E22
:10065E00600874E6254E900046F0E54D600874F093
:10066E00254D900046F0E54EB4010280FE754E0019
:10067E00754D00C2398002C239E54E90384AF828CD
:10068E002873754E00E599B4FF03754D01E599B4D5
:10069E00FE03754D02E599B4FD03754D03E599B45E
:1006AE00FC03754D04E599B4FA03754D05E599B44F
:1006BE00FB06754E01124022E599B4F906754E04FB
:1006CE00124022E599D394E54007E599C394F04092
:1006DE0002801685994F754E027E017F00E54FC34D
:1006EE0094E61266488E328F339007BCE4F0A3F086
:1006FE00E599D394C44007E599C394E64002802857
:10070E0085994F754E0374E5C3954FF533753200D9
:10071E00AE32AF33905F20126617E493F8740193F4
:10072E009007BCC8F0A3C8F0D299020C569000599D
:10073E00E07005A22BB3400280429007BCE0FEA3FE
:10074E00E0FF74FFBE00039F5009EFC39446EE9482
:10075E000640119007BCE0FEA3E0FFEFD3946DEED0
:10076E00940640139007BCE0FEA3E0FF90007812C1
:10077E00666FE599F0800385997480119007BCE04F
:10078E00FEA3E0FF90007812666FE599F09007BC2B
:10079E001266569007BCE0FEA3E0FFEFB40106EE32
:1007AE00B4070280030209FD900778E0B43C028092
:1007BE00030209FDA22B50030208E8C29C900059C7
:1007CE00E0900116F090005AE0900085F090005BEA
:1007DE00E09000A5F090005CE09000CEF090005DFF
:1007EE00E090007AF090005EE09000C0F090005F24
:1007FE00E09000DEF0900060E09000B2F0900061BA
:10080E00E09000D0F0900062E0900100F090006364
:10081E00E0900164F0900064E0900165F090006556
:10082E00E0900166F0123B9490006BE09000E7F0D0
:10083E0090006CE090009EF090006DE090009FF0B4
:10084E0074639007B8F8E4F0E8A3F074AB9000433B
:10085E00F012044E900043E4F07464F5097508003C
:10086E001200E9A2204039757301E573D394075045
:10087E002DE5739007B8F8E4F0E8A3F074AA9000A1
:10088E0043F0120115E573C39407500A7464F50919
:10089E007508001200E97873740126F650CC803783
:1008AE00757308E573D3940E502DE5739007B8F861
:1008BE00E4F0E8A3F074AA900043F0120115E5737A
:1008CE00C3940E500A7464F5097508001200E97895
:1008DE0073740126F650CC0209E7C29C900116E013
:1008EE00900059F0900085E090005AF09000A5E03D
:1008FE0090005BF09000CEE090005CF090007AE00B
:10090E0090005DF09000C0E090005EF09000DEE0A0
:10091E0090005FF09000B2E0900060F09000D0E0A8
:10092E00900061F0900100E0900062F07400900081
:10093E0063F07400900064F07400900065F07463CE
:10094E009007B8F8E4F0E8A3F074AB900043F0120F
:10095E00044E900043E4F07464F50975080012002B
:10096E00E9757301E573D394075026E5739007B8C4
:10097E00F8E4F0E8A3F074AA900043F012011574A5
:10098E0064F5097508001200E97873740126F650B3
:10099E00D3D29C7599FB743C900778F0757308E57B
:1009AE0073D3940E5026E5739007B8F8E4F0E8A3DD
:1009BE00F074AA900043F01201157464F5097508DD
:1009CE00001200E97873740126F650D374C89007AC
:1009DE00B8F8E4F0E8A3F080FE74C89007B8F8E425
:1009EE00F0E8A3F0D29C754E00754D007599FB0290
:1009FE000C569007BCE0FEA3E0FFEF4E7006859903
:100A0E00317530009007BCE0FEA3E0FF74016F4E1D
:100A1E00701BAC30AD31AA32AB33ED2BFBEC3AFA96
:100A2E008A068B0790007812666FE599F09007BCE6
:100A3E001266569007BCE0FEA3E0FF74026F4E7084
:100A4E0021AC30AD3174566D4C7006E54F64E660E6
:100A5E00028003124022123B94854F99754E007509
:100A6E004D00020C569007BCE0FEA3E0FF9000780C
:100A7E0012666FE599F09007BC1266569007BCE0BF
:100A8E00FEA3E0FFAC32AD338F028E038C068D07D2
:100A9E00905F64126617E493F9740193FEEAD39E95
:100AAE00EB994009854F99754E00754D00020C5615
:100ABE009007BCE0FEA3E0FF90007812666FE59908
:100ACE00F09007BC1266569007BCE0FEA3E0FFEF65
:100ADE00B40006EEB401028003020C56900052E000
:100AEE00D394C7400B900052E0C394C8F550801ABF
:100AFE00900052E0D39463400B900052E0C3946494
:100B0E00F5508006900052E0F550E55075F002A4C5
:100B1E00FFAEF08F73EF90007812667AEFFCE0FD77
:100B2E00EC90007B12667AEDFCE0FDEC2DB55002E8
:100B3E008003020C470FEF90007812667AE573FF80
:100B4E00E0FCEF90007C12667AECFFE0FCEFC39CB9
:100B5E00B550028003020C47E57390007A12667A54
:100B6E00E573FFE0FCEF90007D12667AECFFE0FC8F
:100B7E00EF2CB550028003020C47E57390007E12F5
:100B8E00667AE0C39550900059F0E57390007F129D
:100B9E00667AE0C3955090005AF0E573900080128B
:100BAE00667AE0C3955090005BF0740090005CF0A4
:100BBE0074FF90005DF0E57390008212667AE0C3D8
:100BCE00955090005EF0E57390008312667AE0C354
:100BDE00955090005FF0E57390008412667AE0C342
:100BEE009550900060F0E57390008112667AE0C334
:100BFE0095509007B8F8E4F0E8A3F074AB9000437A
:100C0E00F012044E7464F5097508001200E990079D
:100C1E00B812665612044E7464F509750800120077
:100C2E00E99007B812665612044E7599F97464F578
:100C3E00097508001200E980FE7599FF7464F509C4
:080C4E007508001200E980FEA8
:0F384A0002069002073B020A00020A73020ABE3E
:100C560022E54D903859F8282873020D699007BC93
:100C6600E0FEA3E0FF90004812666FE0F59990075A
:100C7600BC1266569007BCE0FEA3E0FF74116F4EEF
:100C86007003754D00020D69856E99020D69900716
:100C9600BCE0FEA3E0FF90007812666FE0F599EFE6
:100CA600B40107EEB40703754D009007BC126656F3
:070CB600020D699007BDE08B
:0F385900020C60020C63020C8E020C94020CB97C
:100CBD00903A0CF8282873855399020D5E855F993B
:100CCD00020D5E856199020D5E856599020D5E8549
:100CDD006799807D85689980788569998073856A23
:100CED0099806E90001AE0F5998066A23AB340079C
:100CFD007599FAC23A8041A22AB3400575990F80C1
:100D0D00359007C7E0600A9007C7E024DCF59980AD
:100D1D00169007C8E0600A9007C8E024DEF59980B8
:100D2D0006900046E0F599900046E4F09007C7E480
:100D3D00F09007C8E4F0C22A8017856B9980128560
:100D4D006699800D856C9980087599FC8003754DA9
:010D5D000095
:103A0C00020CC4020CCA020CD0020CD6020CDC0252
:103A1C000CE1020CE6020CEB020CF0020CF8020DAD
:0D3A2C0047020D4C020D51020D56020D5BBC
:0B0D5E009007BC1266568003123A3961
:03386800020D66E8
:100D690022E537255BFFAE5A50010E9000781266D6
:100D79006FE0F538E537255BFFAE5A50010E0FBF1E
:100D890000010E90007812666FE0F539853F3BE56A
:100D990038B539058538378041E539D39538401D4F
:100DA900E539C39538853AF0A4FFAEF0E53B8E04EA
:100DB9008F05FF126638ED2538F537801DE538C3F4
:100DC9009539853AF0A4FFAEF0E53B8E048F05FF17
:100DD900126638EDF4042538F53722E539D395380C
:100DE900401DE539C39538853AF0A4FFAEF0E53BDF
:100DF9008E048F05FF126638ED2538F537801DE51D
:100E090038C39539853AF0A4FFAEF0E53B8E048FDF
:100E190005FF126638EDF4042538F5372290007E77
:100E2900E0B40170E56775F00A84FF7E008F37E54D
:100E39006775F00A84ADF07C008D3A753F0A755AE2
:100E490005755B24E537C394115005120D6A8006B8
:100E59009005ADE0F537E537900070F0E56775F07E
:100E69000A84FF7E008F37E56775F00A84ADF07C50
:100E7900008D3A753F0A755A05755B5AE537C39473
:100E8900115005120D6A80069005E3E0F537E53744
:100E9900900012F02290007EE0B4016AE56775F0D7
:100EA9000A84FF7E008F37E56775F00A84ADF07C10
:100EB900008D3A753F0A755A05755B36E537C39457
:100EC900115005120D6A80069005BFE0F537853788
:100ED9004BE56775F00A84FF7E008F37E56775F08B
:100EE9000A84ADF07C008D3A753F0A755A05755B29
:100EF90048E537C394115005120D6A80069005D153
:100F0900E0F53785374C22E55F75F00484FF7E00F4
:100F19008F37E55F75F00484ADF07C008D3A753F3D
:100F290004755A01755B00E537C3943F5005120DEE
:100F39006A80069001B7E0F5378537297528009052
:100F49000045E075F020A4FFAEF09000C9E08E04E2
:100F59008F05FF1266388D379000B1E0D3955F5049
:100F6900030210169000D5E0D3955F4010ED900173
:100F7900B812667AE0F52B752A000210139000A0CA
:100F8900E0D3955F4043E5379001B812667AE0F502
:100F990038E5379001D812667AE0F5399000D5E046
:100FA900F404255FF53A9000A0E0FE9000D5E0F446
:100FB900042EF53BE538B539058538378003120D20
:100FC900E485372B752A008041E5379001D81266F0
:100FD9007AE0F538E5379001F812667AE0F539904C
:100FE90000A0E0F404255FF53A9000B1E0FE90001E
:100FF900A0E0F4042EF53BE538B53905853837808E
:1010090003120DE485372B752A000210BD9000D814
:10101900E0D3955F5011E53790023812667AE0F512
:101029002B752A000210BD9000A1E0D3955F5043B3
:10103900E53790021812667AE0F538E537900238FC
:1010490012667AE0F5399000A1E0F404255FF53ADB
:101059009000D8E0FE9000A1E0F4042EF53BE538BD
:10106900B539058538378003120DE485372B752A84
:10107900008041E5379001F812667AE0F538E537E6
:1010890090021812667AE0F5399000B1E0F404256F
:101099005FF53A9000A1E0FE9000B1E0F4042EF56E
:1010A9003BE538B539058538378003120DE48537B6
:1010B9002B752A00229000E9E0F53C753F11755A1D
:1010C90002755B00AE52AF53E53C75F00FA4FDAC61
:1010D900F0EDD39FEC9E4021E53C8E048F05FF1275
:1010E9006638ED75F010A4FFAEF0E55F75F0118478
:1010F900FD7C00ED2FF53D800EE55F75F01184FF55
:101109007E00EF24F0F53D853D37E55F75F01184EC
:10111900AFF07E008F3A120D6A85373EAE52AF535B
:101129009000E9E075F00FA4FDACF0EDD39FEC9EC3
:101139004028755A02755B10853D37120D6A853E48
:1011490038853739AE52AF53E53C8E048F05FF120F
:1011590066638D3A853C3B120DE485372975280075
:10116900752B64752A00229000E9E0F53C753F1162
:10117900755A02755B00AE52AF53E53C75F00FA48A
:10118900FDACF0EDD39FEC9E4021E53C8E048F052C
:10119900FF126638ED75F010A4FFAEF0E56175F049
:1011A9001184FD7C00ED2FF53D800EE56175F01190
:1011B90084FF7E00EF24F0F53D853D37E56175F04C
:1011C9001184AFF07E008F3A120D6A85373EAE5218
:1011D900AF539000E9E075F00FA4FDACF0EDD39F9B
:1011E900EC9E4028755A02755B10853D37120D6AD1
:1011F900853E38853739AE52AF53E53C8E048F05AD
:10120900FF1266638D3A853C3B120DE485372975DB
:101219002800E56B6017E56BC394FE50109000DD64
:10122900E0B402099000CBE0D3940B50028017AED2
:1012390028AF29E56B12664874E78E048F05FF1203
:1012490066388C288D299000B3E0B40453E55F75A6
:10125900F00484FF7E008F37E55F75F00484ADF0FC
:101269007C008D3A753F04755A01755B00E537C3FB
:10127900943F5005120D6A80069001B7E0F537AE2C
:1012890028AF29E53712664874648E048F05FF126A
:101299006638AE28AF29EF2DFDEE3CFC8C288D2950
:1012A900752B64752A002290007EE0B40146E5673B
:1012B90075F00A84FF7E008F37E56775F00A84AD03
:1012C900F07C008D3A753F0A755A05755B00E53764
:1012D900C394115005120D6A8006900589E0F5370F
:1012E900AE2AAF2BE5372FFF50010E746412668CBE
:1012F9008E2A8F2B90007FE0B40146E56875F00ACD
:1013090084FF7E008F37E56875F00A84ADF07C00B4
:101319008D3A753F0A755A05755B6CE537C39411AB
:101329005005120D6A80069005F5E0F537AE2AAF33
:101339002BE5372FFF50010E746412668C8E2A8FAD
:101349002B90008EE0B40249E56AC3944175F0051B
:1013590084FF7E008F37E56A75F00584ADF07C0067
:101369008D3A753F05755A06755B00E537C39413C9
:101379005005120D6A800690068BE0F537AE2AAF4C
:101389002BE5372FFF50010E746412668C8E2A8F5D
:101399002B9000D0E0B40202800302144FE55F7580
:1013A900F01584FF7E008F37E55F75F01584ADF089
:1013B9007C008D3A753F15755A03755BF4E537C3A3
:1013C900940B5005120D6A8006900477E0F537E515
:1013D9003775F0FFA4FFAEF09000D1E08E048F05C1
:1013E900FF126638ED900069F0E56675F078A4FFA4
:1013F900AEF074FF8E048F05FF1266388C5A8D5B30
:1014090074028C068D071200398F37AC5AAD5B74A4
:1014190004FF1266638D3A753F04755A06755B2899
:10142900E537C3941D5005120D6A80069006BDE08C
:10143900F537AE2AAF2BE5372FFF50010E74641232
:10144900668C8E2A8F2B90007DE0B4025DE5617574
:10145900F064A4FFAEF074081200398E5C8F5D74DD
:10146900058E048F05FF1266388D37AE5CAF5D744B
:10147900058E048F05FF1266638D3A753F05755A0F
:1014890005755BDEE537C394135005120D6A8006B6
:10149900900669E0F537AE2AAF2BE5372FFF5001EB
:1014A9000E746412668C8E2A8F2B9000BFE0703CFC
:1014B900900045E075F00584FF7E008F3790004568
:1014C900E075F00584ADF07C008D3A753F05755ADD
:1014D90005755BC0E537C3941D5005120D6A80067A
:1014E900900655E0F537E537900071F022900086B7
:1014F900E0B401179007C3E0252BFFAE2A50010E77
:101509009000DAE012668C8E2A8F2B9000FEE0B4F0
:1015190001149000FFE0A852B8000495535007E564
:101529005FC39560400280129000A8E0252BFFAEB2
:101539002A50010E8E2A8F2B802F900086E0B4034B
:1015490016A22DB3B350109007C6E0C39405A85254
:10155900B800069553400280109000A8E0252BFFA3
:10156900AE2A50010E8E2A8F2B900080E0B4020221
:1015790080030218F4900083E0602FE567D3944656
:101589004028900013E0FEA3E0FF9000BEE075F054
:1015990003A4FDACF0EFD39DEE9C400E9000E2E079
:1015A900A852B80005D3955350030218F49000B31C
:1015B900E0B40302800302175885615B755A0090F5
:1015C900008AE0A852B800049553500E90008BE0B1
:1015D900A85AB80005D3955B5003021755E5617504
:1015E900F002A4FFAEF074158E048F05FF12663861
:1015F9008C068D0790060812666FFEE0FFEE9000DC
:1016090082E0FEEF8E0088F0A4FFAEF074648E04D1
:101619008F05FF1266388C5A8D5B900045E075F096
:1016290018A4FFAEF09000C9E08E048F05FF126682
:10163900388C068D0790062012666FAE5AAF5BE0B4
:1016490012664874648E048F05FF1266388C5A8DB1
:101659005BE565A85AB80077D3955B4072E565C329
:10166900955BFFE4955AFE8E5A8F5B7428BE000382
:101679009F500C755B28755A00740D900046F0AEAA
:101689005AAF5B900083E012664874288E048F0578
:10169900FF1266388C5A8D5BAE28AF29740A8E0406
:1016A9008F05FF1266388D068C07AC5AAD5BCFCE1D
:1016B900CF120003740A8E048F05FF1266388C5A04
:1016C9008D5BAE28AF291266948E288F29807DE51F
:1016D90065A85AB80004955B5072AE5AAF5BE565D0
:1016E90012668C8E5A8F5B7428BE00039F500C754E
:1016F9005B28755A00740D900046F0AE5AAF5B90A6
:101709000083E012664874288E048F05FF1266383C
:101719008C5A8D5BAE28AF29740A8E048F05FF128F
:1017290066388D068C07AC5AAD5BCFCECF1200035D
:10173900740A8E048F05FF1266388C5A8D5BAE28A9
:10174900AF29EF2DFDEE3CFC8C288D290218F49071
:1017590000CBE0855FF0A4FFAEF074051266487413
:10176900071200398E5A8F5B90008AE0A852B800A0
:10177900049553501290008BE075F002A4FDACF073
:10178900EFC39DEE9C40030218F4E55F75F00B84EE
:10179900FF7E0090060812666FFEE0FFEE90008261
:1017A900E0FEEF8E0088F0A4FFAEF074648E048F23
:1017B90005FF1266388C5A8D5B900045E075F0186C
:1017C900A4FFAEF09000C9E08E048F05FF126638C1
:1017D9008C068D0790062012666FAE5AAF5BE01239
:1017E900664874648E048F05FF1266388C5A8D5BC7
:1017F900E565A85AB80077D3955B4072E565C3954E
:101809005BFFE4955AFE8E5A8F5B7428BE00039FD6
:10181900500C755B28755A00740D900046F0AE5A4D
:10182900AF5B900083E012664874288E048F05FF31
:101839001266388C5A8D5BAE28AF29740A8E048FD4
:1018490005FF1266388D068C07AC5AAD5BCFCECF3B
:10185900120003740A8E048F05FF1266388C5A8DA4
:101869005BAE28AF291266948E288F29807DE565A5
:10187900A85AB80004955B5072AE5AAF5BE5651281
:10188900668C8E5A8F5B7428BE00039F500C755B63
:1018990028755A00740D900046F0AE5AAF5B90005F
:1018A90083E012664874288E048F05FF1266388C0F
:1018B9005A8D5BAE28AF29740A8E048F05FF126614
:1018C900388D068C07AC5AAD5BCFCECF12000374AE
:1018D9000A8E048F05FF1266388C5A8D5BAE28AFCD
:1018E90029EF2DFDEE3CFC8C288D29229000DEE0AD
:1018F900B4026AE55F75F00884FF7E008F37E55F03
:1019090075F00884ADF07C008D3A753F08755A0171
:10191900755BE0E537C3943F5005120D6A80069068
:101929000277E0F53785372D752C00AE2CAF2DAC3D
:101939002AAD2B12000374648E048F05FF126638DA
:101949008C2C8D2D90007BE08C068D0712664874D7
:10195900648E048F05FF1266388C2C8D2DAE28AF4E
:1019690029AC2AAD2B12000374648E048F05FF1273
:1019790066388C288D2990007BE08C068D071266CD
:101989004874648E048F05FF1266388C288D29A24D
:101999000D401DAE52AF537405BE00039F5002D2D5
:1019A9000DE561D394CC4008D2017411900046F042
:1019B9009000DDE0B402089000CBE0640B60028087
:1019C90035AE28AF29E56B12664874E78E048F059A
:1019D900FF1266388C288D299000DEE0B40217AE1C
:1019E9002CAF2DE56B12664874E78E048F05FF1244
:1019F90066388C2C8D2D90009DE05402601B900060
:101A090094E0A852B80012D39553400DA20DB3B378
:101A19005007E561C3949A40028028AE34AF3590EF
:101A29000092E075F002A4FDACF0EF2DFDEE3CFC58
:101A390074022DFD50010CE561BC0007D39D4003E4
:101A4900754301856135753400E5437003021B3820
:101A59009000F0E0C395435003021B2A900100E077
:101A6900C394025076E56775F00A84FF7E009005FD
:101A79007812666FE0F55B755A00AE5AAF5B90005D
:101A890093E012664874648E048F05FF1266388CE1
:101A99005C8D5D9000F0E004C395438C068D0712C0
:101AA90066489000F0E08E048F05FF1266388C5C62
:101AB9008D5DAE28AF29EF2DFDEE3CFC8C288D29DC
:101AC9009000DEE0B40212AE2CAF2DAA5CAB5DEF44
:101AD9002BFBEE3AFA8A2C8B2D80469000F0E0041D
:101AE900C39543854BF0A4FFAEF09000F0E08E045F
:101AF9008F05FF1266388C5C8D5DAE28AF29EF2DFE
:101B0900FDEE3CFC8C288D299000DEE0B40212AE7B
:101B19002CAF2DAA5CAB5DEF2BFBEE3AFA8A2C8B2E
:101B29002D05439000F0E0C39543500375430090A1
:101B3900009DE05401601B900091E0A852B800128A
:101B4900D39553400DA20DB3B35007E55FC394CCB1
:101B59004002802590008FE075F003A4FFAEF0E508
:101B6900402FFF50010E74032FFF50010EE55FBE99
:101B79000007D39F4003754401855F40E544700326
:101B8900021C6B9000F1E0C395445003021C5D9068
:101B99000100E0C394025076E56775F00A84FF7E80
:101BA9000090057812666FE0F55B755A00AE5AAF82
:101BB9005B900090E012664874648E048F05FF12F2
:101BC90066388C5C8D5D9000F1E004C395448C0609
:101BD9008D071266489000F1E08E048F05FF1266AA
:101BE900388C5C8D5DAE28AF29EF2DFDEE3CFC8C69
:101BF900288D299000DEE0B40212AE2CAF2DAA5C2C
:101C0900AB5DEF2BFBEE3AFA8A2C8B2D80469000C8
:101C1900F1E004C39544854CF0A4FFAEF09000F1C7
:101C2900E08E048F05FF1266388C5C8D5DAE28AF9F
:101C390029EF2DFDEE3CFC8C288D299000DEE0B4C7
:101C49000212AE2CAF2DAA5CAB5DEF2BFBEE3AFA7C
:101C59008A2C8B2D05449000F1E0C39544500375FF
:101C690044009000F3E02529FFAE2850010E8E288C
:101C79008F299000A2E0A828B8000495295009905E
:101C890000A2E0F5297528009000DEE0B4020D906D
:101C990000A2E0A82CB80006952D4002800990000A
:101CA900A2E0F52D752C00229000DEE0B40102803F
:101CB90003021DBCA20DB35003021DBA9000A9E096
:101CC900B40168AE28AF29AC52AD53120003743C7D
:101CD9008E048F05FF1266389000B9E0BC00109D94
:101CE900400D9000BBE0A828B8000495295002D205
:101CF90002AE28AF29AC52AD53120003743C8E04D6
:101D09008F05FF1266389000B9E0C3940ABC00152C
:101D1900D39D40119000BBE0C39405A828B80005E5
:101D2900D3952950028002C2028068AE28AF29AC3F
:101D390052AD5312000374788E048F05FF12663872
:101D49009000B9E0BC00109D400D9000BBE0A828B0
:101D5900B8000495295004D2028038AE28AF29ACC6
:101D690052AD5312000374788E048F05FF12663842
:101D79009000B9E0C3940ABC0015D39D40119000AE
:101D8900BBE0C39405A828B80005D3952950028063
:101D990002C202A202B34019AE28AF299000BAE0EC
:101DA90012664874648E048F05FF1266388C288D7C
:101DB900298002C202A200B34006A201B3B35009AE
:101DC900900019E4F0A3F08024AE28AF297400D361
:101DD9009F74019E400C900019E528F0A3E529F0B5
:101DE900800B74FF900019F8E4F0E8A3F09000C0AC
:101DF900E0D39402400C9000ABE07006A20DB3B39F
:101E09004002801AAE28AF2974021266488E288FC4
:101E190029AE2CAF2D74021266488E2C8F2D90009E
:101E2900A9E0B4011AAE28AF2974021266488E28B7
:101E39008F29AE2CAF2D74021266488E2C8F2DAED1
:101E490028AF29745E126648740A8E048F05FF1242
:101E590066388C288D299000DEE0B40217AE2CAFCD
:101E69002D745E126648740A8E048F05FF12663857
:101E79008C2C8D2DAE28AF297402BE000AD39F4049
:101E890006752902752800AE2CAF2D7402BE000A12
:101E9900D39F4006752D02752C00900017E528F098
:101EA900A3E529F022900045E090037812667AE0D4
:101EB900F541754264900045E0FE9000B4E0D39E80
:101EC9004037E55F75F00884FF7E008F37E55F7561
:101ED900F00884ADF07C008D3A753F08755A03759A
:101EE9005B96E537C3941F5005120D6A800690046E
:101EF9002DE0F5378537428035E55F75F00884FFB9
:101F09007E008F37E55F75F00884ADF07C008D3A6F
:101F1900753F08755A03755BB6E537C3941F5005BD
:101F2900120D6A800690044DE0F5378537422290FC
:101F390000EAE0F53C753F11755A04755B00AE5235
:101F4900AF53E53C75F00FA4FDACF0EDD39FEC9ECB
:101F59004021E53C8E048F05FF126638ED75F010BF
:101F6900A4FFAEF0E55F75F01184FD7C00ED2FF55F
:101F79003D800EE55F75F01184FF7E00EF24F0F5DA
:101F89003D853D37E55F75F01184AFF07E008F3AEE
:101F9900120D6A85373EAE52AF539000EAE075F0F4
:101FA9000FA4FDACF0EDD39FEC9E4028755A047543
:101FB9005B10853D37120D6A853E38853739AE523B
:101FC900AF53E53C8E048F05FF1266638D3A853C5D
:101FD9003B120DE4853741754264229000EAE0F531
:101FE9003C753F11755A04755B00AE52AF53E53C21
:101FF90075F00FA4FDACF0EDD39FEC9E4021E53CBC
:102009008E048F05FF126638ED75F010A4FFAEF04F
:10201900E56175F01184FD7C00ED2FF53D800EE53D
:102029006175F01184FF7E00EF24F0F53D853D37A1
:10203900E56175F01184AFF07E008F3A120D6A8563
:10204900373EAE52AF539000EAE075F00FA4FDACF5
:10205900F0EDD39FEC9E4028755A04755B10853DC1
:1020690037120D6A853E38853739AE52AF53E53C94
:102079008E048F05FF1266638D3A853C3B120DE491
:102089008537417542649000B3E0B4047990004506
:10209900E0FE9000B4E0D39E4037E55F75F0088418
:1020A900FF7E008F37E55F75F00884ADF07C008D09
:1020B9003A753F08755A03755B96E537C3941F5007
:1020C90005120D6A800690042DE0F53785374280A8
:1020D90035E55F75F00884FF7E008F37E55F75F0A1
:1020E9000884ADF07C008D3A753F08755A03755B1D
:1020F900B6E537C3941F5005120D6A800690044D4A
:10210900E0F5378537422290007EE0B4013BE56770
:1021190075F00A84FF7E008F37E56775F00A84AD94
:10212900F07C008D3A753F0A755A05755B12E537E3
:10213900C394115005120D6A800690059BE0F5378E
:10214900E5422537C39464F54290007FE0B4013B32
:10215900E56875F00A84FF7E008F37E56875F00A37
:1021690084ADF07C008D3A753F0A755A05755B7E22
:10217900E537C394115005120D6A8006900607E0F1
:10218900F537E5422537C39464F542E5412542F523
:1021990036900086E0B402109007C2E02536FE9022
:1021A90000DAE0F4042EF5369000DDE0D394014026
:1021B90040E56BC394E7501D74E7C3956BFE900728
:1021C900C4E08E00F5F0E884FF7E008F37E5362500
:1021D90037F536801CE56BC394E7FE9007C4E08EA3
:1021E90000F5F0E884FF7E008F37E536C39537F5B3
:1021F90036A20D4006E5412464F536E536D39464EC
:102209004009E536C39464F53680037536009000BD
:10221900B6E0C3953650069000B6E0F53622D200F6
:1022290090006FE0A852B800049553504190006F98
:10223900E0A852B800049553500375360F90006F0B
:10224900E004A852B800049553500375360A90006B
:102259006FE02402A852B80004955350057536055D
:10226900C20090006FE060067409900046F0C23D1C
:102279007E017F009000BCE01266489000CBE08EA2
:10228900048F05FF126638E55FBC0017D39D401324
:102299009000C5E0B40204D23D8002C200740A90E5
:1022A9000046F09000BDE0C3956750159000CFE05F
:1022B900A852B8000495535002C200740B9000460E
:1022C900F0E567C39464501D900115E0600D90011D
:1022D90015E0A852B80006955340028008C2007460
:1022E9000B900046F0A20040037536059000FEE011
:1022F900B401149000FFE0A852B8000495535007A8
:10230900E55FC39560400280089000A7E0F536803C
:102319003A900086E0B40306A22DB3B34002802BA5
:102329009007C6E0C39405A852B800049553500C11
:102339009000A7E0F536740C900046F09007C6E0CF
:10234900A852B8000495535002C20085366C90001B
:1023590078E02536FE900045E075F01E84FC7F008C
:10236900EE2CF53622900045E075F00584FF7E00DD
:102379008F37900045E075F00584ADF07C008D3A0B
:10238900753F05755A03755BD69000C9E01475F061
:102399000584FF7E00E537BE00039F5005120D6AD4
:1023A900800BE53790044E12667AE0F537E53790F1
:1023B90007C5F09007C5E0FE9000B8E0C39E50083D
:1023C9009000B8E09007C5F022E56775F00A84FF30
:1023D9007E0090057812666FE0F546E546D3946471
:1023E9004010E546C3946475F00F84FF7E008F4664
:1023F900800375460090009BE02546F54622900033
:10240900B3E0C3940350269007B2E0FEA3E0FF7443
:1024190004120039E55F126648740F8E048F05FFB8
:102429001266389007B0ECF0A3EDF080249007B263
:10243900E0FEA3E0FF7404120039E56112664874F6
:102449000F8E048F05FF1266389007B0ECF0A3EDEC
:10245900F090008EE0B40262E56AC3944175F0051C
:1024690084FF7E008F37E56A75F00584ADF07C0046
:102479008D3A753F05755A06755B14E537C3941790
:102489005005120D6A800690069FE0F5379007B057
:10249900E0FEA3E0FF740A8E048F05FF126638E59B
:1024A900378C068D07126648740A8E048F05FF1251
:1024B90066389007B0ECF0A3EDF09007B0E0FEA30A
:1024C900E0FF9007B6E0FCA3E0FDEDD39FEC9E4052
:1024D9000F9007B6E0F8A3E09007B0C8F0A3C8F0E2
:1024E900229006BFE090386BF8282873804C8553FA
:1024F9007380479000CBE0855FF0A4FFAEF07408CD
:102509001200398F738033856173802E85677380DC
:10251900298568738024856973801F856A73801A89
:10252900856B7380158566738010856573800B854F
:0A2539006C73800690001AE0F57341
:10386B000224F50224F70224FC022510022515027E
:10387B00251A02251F02252402252902252E0225A1
:07388B003302253802253D40
:102543009006C0E0FE9006C1E0D39E404B9006BFCC
:10255300E0B404189006C1E0C395735002D22E90E4
:1025630006C0E0D395734002C22E802A9006C0E0D5
:10257300C3957350099006C1E0D39573500280024E
:10258300D22E9006C0E0D3957350099006C1E0C3E4
:1025930095735002C22E802A9006C0E0D3957340F3
:1025A300099006C1E0C3957340028002C22E9006D3
:1025B300C0E0C3957340099006C1E0D39573400210
:1025C300D22E229006C3E0903892F8282873804CCC
:1025D30085537380479000CBE0855FF0A4FFAEF096
:1025E30074081200398F738033856173802E856779
:1025F3007380298568738024856973801F856A7356
:10260300801A856B7380158566738010856573806A
:0C2613000B856C73800690001AE0F573D4
:103892000225D10225D30225D80225EC0225F10208
:1038A20025F60225FB02260002260502260A02262A
:0738B2000F02261402261983
:10261F009006C4E0FE9006C5E0D39E405F9006C3CF
:10262F00E0B404189006C5E0C395735002D22F9002
:10263F0006C4E0D395734002C22F803E9006C4E0DB
:10264F00C3957350099006C5E0D39573500280026D
:10265F00D22F9006C4E0D3957350099006C5E0C3FE
:10266F0095735002C22F9006C3E0B401099000D7B2
:10267F00E0D3956150028002C22F802A9006C4E0F9
:10268F00D3957340099006C5E0C39573400280024D
:10269F00C22F9006C4E0C3957340099006C5E0D3DE
:1026AF0095734002D22F229006C7E09038B9F828D0
:1026BF002873804C85537380479000CBE0855FF083
:1026CF00A4FFAEF074081200398F738033856173E5
:1026DF00802E856773802985687380248569738050
:1026EF001F856A73801A856B7380158566738010DA
:1026FF00856573800B856C73800690001AE0F57307
:1038B9000226C10226C30226C80226DC0226E1022C
:1038C90026E60226EB0226F00226F50226FA022651
:0738D900FF0227040227098A
:10270F009006C8E0FE9006C9E0D39E404B9006C7E6
:10271F00E0B404189006C9E0C395735002D230900C
:10272F0006C8E0D395734002C230802A9006C8E0F5
:10273F00C3957350099006C9E0D395735002800278
:10274F00D2309006C8E0D3957350099006C9E0C304
:10275F0095735002C230802A9006C8E0D39573401B
:10276F00099006C9E0C3957340028002C2309006FB
:10277F00C8E0C3957340099006C9E0D39573400232
:10278F00D230229006CBE09038E0F8282873804CA6
:10279F0085537380479000CBE0855FF0A4FFAEF0C8
:1027AF0074081200398F738033856173802E8567AB
:1027BF007380298568738024856973801F856A7388
:1027CF00801A856B7380158566738010856573809D
:0C27DF000B856C73800690001AE0F57307
:1038E00002279D02279F0227A40227B80227BD02B4
:1038F00027C20227C70227CC0227D10227D60227D8
:07390000DB0227E00227E5CE
:1027EB009006CCE0FE9006CDE0D39E404B9006CBFE
:1027FB00E0B404189006CDE0C395735002D231902B
:10280B0006CCE0D395734002C231802A9006CCE00F
:10281B00C3957350099006CDE0D395735002800297
:10282B00D2319006CCE0D3957350099006CDE0C31E
:10283B0095735002C231802A9006CCE0D395734039
:10284B00099006CDE0C3957340028002C231900619
:10285B00CCE0C3957340099006CDE0D3957340024D
:10286B00D231229006CFE0903907F8282873804C9C
:10287B0085537380479000CBE0855FF0A4FFAEF0EB
:10288B0074081200398F738033856173802E8567CE
:10289B007380298568738024856973801F856A73AB
:1028AB00801A856B738015856673801085657380C0
:0C28BB000B856C73800690001AE0F5732A
:1039070002287902287B022880022894022899023B
:10391700289E0228A30228A80228AD0228B202285E
:07392700B70228BC0228C111
:1028C7009006D0E0FE9006D1E0D39E404B9006CF15
:1028D700E0B404189006D1E0C395735002D2329049
:1028E70006D0E0D395734002C232802A9006D0E02A
:1028F700C3957350099006D1E0D3957350028002B7
:10290700D2329006D0E0D3957350099006D1E0C338
:1029170095735002C232802A9006D0E0D395734057
:10292700099006D1E0C3957340028002C232900637
:10293700D0E0C3957340099006D1E0D39573400268
:10294700D232229006D3E090392EF8282873804C93
:1029570085537380479000CBE0855FF0A4FFAEF00E
:1029670074081200398F738033856173802E8567F1
:102977007380298568738024856973801F856A73CE
:10298700801A856B738015856673801085657380E3
:0C2997000B856C73800690001AE0F5734D
:10392E0002295502295702295C02297002297502C3
:10393E00297A02297F02298402298902298E0229E5
:07394E009302299802299D54
:1029A3009006D4E0FE9006D5E0D39E404B9006D32C
:1029B300E0B404189006D5E0C395735002D2339067
:1029C30006D4E0D395734002C233802A9006D4E044
:1029D300C3957350099006D5E0D3957350028002D6
:1029E300D2339006D4E0D3957350099006D5E0C353
:1029F30095735002C233802A9006D4E0D395734076
:102A0300099006D5E0C3957340028002C233900655
:102A1300D4E0C3957340099006D5E0D39573400283
:102A2300D233229006D7E0903955F8282873804C8A
:102A330085537380479000CBE0855FF0A4FFAEF031
:102A430074081200398F738033856173802E856714
:102A53007380298568738024856973801F856A73F1
:102A6300801A856B73801585667380108565738006
:0C2A73000B856C73800690001AE0F57370
:10395500022A31022A33022A38022A4C022A51024B
:103965002A56022A5B022A60022A65022A6A022A6C
:073975006F022A74022A7997
:102A7F009006D8E0FE9006D9E0D39E404B9006D743
:102A8F00E0B404189006D9E0C395735002D2349085
:102A9F0006D8E0D395734002C234802A9006D8E05E
:102AAF00C3957350099006D9E0D3957350028002F5
:102ABF00D2349006D8E0D3957350099006D9E0C36D
:102ACF0095735002C234802A9006D8E0D395734094
:102ADF00099006D9E0C3957340028002C234900674
:102AEF00D8E0C3957340099006D9E0D3957340029F
:102AFF00D234229006DBE090397CF8282873804C82
:102B0F0085537380479000CBE0855FF0A4FFAEF054
:102B1F0074081200398F738033856173802E856737
:102B2F007380298568738024856973801F856A7314
:102B3F00801A856B73801585667380108565738029
:0C2B4F000B856C73800690001AE0F57393
:10397C00022B0D022B0F022B14022B28022B2D02D3
:10398C002B32022B37022B3C022B41022B46022BF3
:07399C004B022B50022B55DA
:102B5B009006DCE0FE9006DDE0D39E404B9006DB5A
:102B6B00E0B404189006DDE0C395735002D23590A3
:102B7B0006DCE0D395734002C235802A9006DCE078
:102B8B00C3957350099006DDE0D395735002800214
:102B9B00D2359006DCE0D3957350099006DDE0C387
:102BAB0095735002C235802A9006DCE0D3957340B2
:102BBB00099006DDE0C3957340028002C235900692
:102BCB00DCE0C3957340099006DDE0D395734002BA
:102BDB00D235229006DFE09039A3F8282873804C79
:102BEB0085537380479000CBE0855FF0A4FFAEF078
:102BFB0074081200398F738033856173802E85675B
:102C0B007380298568738024856973801F856A7337
:102C1B00801A856B7380158566738010856573804C
:0C2C2B000B856C73800690001AE0F573B6
:1039A300022BE9022BEB022BF0022C04022C09025E
:1039B3002C0E022C13022C18022C1D022C22022C7A
:0739C30027022C2C022C311D
:102C37009006E0E0FE9006E1E0D39E404B9006DF71
:102C4700E0B404189006E1E0C395735002D23690C1
:102C570006E0E0D395734002C236802A9006E0E092
:102C6700C3957350099006E1E0D395735002800233
:102C7700D2369006E0E0D3957350099006E1E0C3A1
:102C870095735002C236802A9006E0E0D3957340D0
:102C9700099006E1E0C3957340028002C2369006B0
:102CA700E0E0C3957340099006E1E0D395734002D5
:102CB700D236229006E3E09039CAF8282873804C70
:102CC70085537380479000CBE0855FF0A4FFAEF09B
:102CD70074081200398F738033856173802E85677E
:102CE7007380298568738024856973801F856A735B
:102CF700801A856B73801585667380108565738070
:0C2D07000B856C73800690001AE0F573D9
:1039CA00022CC5022CC7022CCC022CE0022CE502E8
:1039DA002CEA022CEF022CF4022CF9022CFE022D06
:0739EA0003022D08022D0D60
:102D13009006E4E0FE9006E5E0D39E404B9006E388
:102D2300E0B404189006E5E0C395735002D23790DF
:102D330006E4E0D395734002C237802A9006E4E0AC
:102D4300C3957350099006E5E0D395735002800252
:102D5300D2379006E4E0D3957350099006E5E0C3BB
:102D630095735002C237802A9006E4E0D3957340EE
:102D7300099006E5E0C3957340028002C2379006CE
:102D8300E4E0C3957340099006E5E0D395734002F0
:102D9300D23722AE2EAF2F74F5D39F74019E400815
:102DA300782E12669C022EB0752F01752E00AE523E
:102DB300AF53E546BE000DD39F40099000ADE0D36D
:102DC300954740028023754700E546C39553F57345
:102DD3009000B0E0D395454008E5452573F545805F
:102DE300069000B0E0F54580020547900089E0D3E6
:102DF3009561401CE55FC395604015AE52AF53E546
:102E030046BE00039F50099000AEE0D395484002B0
:102E1300806E9007C9E0A852B8000495535003751B
:102E23004A009007C9E0A852B8000BD39553400657
:102E3300E5539007C9F0E54A7041E553C39546F55C
:102E430073E573D3940540037573059000AFE0C336
:102E530095455007E573C3954540028009E545C391
:102E63009573F54580069000AFE0F5459000AFE01F
:102E7300D3954540069000AFE0F5457548008002C4
:102E83000548E54A7016900089E0C39561500DE549
:102E9300462405A852B8000695534002800F9000BF
:102EA3009CE0F545754A0174789007C9F022AE2E6F
:102EB300AF2F74E9D39F74039E4008782E12669C4B
:102EC30002304F752F01752E00754532A238402A06
:102ED30075451990009CE075F002A4FFAEF0E5473C
:102EE300BE0006D39F4002D2380547754A03747863
:102EF3009007C9F075490002303EAE52AF53E54624
:102F03006F4E700302303EE546BE000DD39F40096D
:102F13009000ADE0D395474002800F754700E54A26
:102F2300C394035003754519800DE546C39553F5C6
:102F330073E5472573F547900089E0D39561400E0B
:102F43009007C9E0A852B80007D395534002800CFC
:102F5300054990009CE0B54903754A00E54AB4036E
:102F630006A20DB3B34002800A0549E549B43C0308
:102F7300754A02E54AB402299007C9E0A852B8008D
:102F83000ED395534009E5539007C9F07549009056
:102F93000089E0C39561500975490074789007C9A9
:102FA300F0E54A705A900089E0D39561401CE55FD3
:102FB300C395604015AE52AF53E546BE00039F5024
:102FC300099000AEE0D3954840028008754800752B
:102FD300454B8028E553C39546F573E573D39405B4
:102FE3004003757305900089E0D395614008E54877
:102FF3002573F5488006E5482406F548754900E53C
:103003004A7016900089E0C39561500DE54624058A
:10301300A852B80006955340028003754A01E54A59
:10302300B40118754519054990009CE0B54906752A
:103033004A0275490074789007C9F0E54575F00AAE
:10304300A4FFAEF09007BAEEF0A3EFF022E56F9085
:1030530039F1F8282873900081E0700302327790E9
:1030630000B7E0B401028003023192900044E0B55E
:103073005E02800302318F7E017F00E5BE12664847
:10308300E5BD2FFF50010E8E5A8F5B7410126648F8
:1030930090006EE08E048F05FF1266389007BEEC39
:1030A300F0A3EDF074FFBC00039D500B74FF900779
:1030B300BEF8E4F0E8A3F0E56B600FE56BC394FEA4
:1030C30050089000DDE06402600280649000CBE071
:1030D300B40B1F9007BEE0FEA3E0FF74E71266483F
:1030E300E56B8E048F05FF1266389007BEECF0A3E4
:1030F300EDF09000CBE0D3940B40089000B3E06474
:10310300046002802B9007BEE0FEA3E0FF9007C09F
:10311300E0FCA3E0FDEFD39DEE9C400D126694907E
:1031230007BEEEF0A3EFF080079007BEE4F0A3F034
:10313300900081E0B4021E9007BEE0FEA3E0FF9082
:1031430007CAE02FFF50010E74011200399007BE29
:10315300EEF0A3EFF09007BEE0FEA3E0FF9007CAF6
:10316300E0BE0008D39F4004D23B8002B23B9007ED
:10317300BFE09007CAF09000B3E064016006A23B91
:10318300B3B3400280069007BFE0F55F023275D209
:103193003B7E017F00E5BE126648E5BD2FFF50016F
:1031A3000E8E5A8F5B741012664890006EE08E0488
:1031B3008F05FF1266389007BEECF0A3EDF0E56BC8
:1031C300600FE56BC394FE50089000DDE06402607D
:1031D3000280649000CBE0B40B1F9007BEE0FEA317
:1031E300E0FF74E7126648E56B8E048F05FF1266F5
:1031F300389007BEECF0A3EDF09000CBE0D3940B36
:1032030040089000B3E064046002802B9007BEE0A6
:10321300FEA3E0FF9007C0E0FCA3E0FDEFD39DEE2B
:103223009C400D1266949007BEEEF0A3EFF080076A
:103233009007BEE4F0A3F0900081E0B4021E900773
:10324300BEE0FEA3E0FF9007CAE02FFF50010E741B
:10325300011200399007BEEEF0A3EFF09007BFE034
:103263009007CAF09000B3E0640160069007BFE0E6
:10327300F55F8003755F0090007DE07006756F0158
:1032830002305075BB1802384590007DE070030290
:1032930033FD7E017F00E5BE126648E5BD2FFF507A
:1032A300010E8E5A8F5B9000C3E0B4010F7E0F7F37
:1032B300FFAC5AAD5B1266948E5A8F5B9000E8E0C8
:1032C300B40245AE5AAF5B900023E0FCA3E0FDEDF2
:1032D300D39FEC9E400A900023E55AF0A3E55BF0F0
:1032E300AE5AAF5B900025E0FCA3E0FDEFD39DEE6B
:1032F3009C400A900025E55AF0A3E55BF0AE5AAF77
:103303005B74041200398F619000E8E0704CAE5A90
:10331300AF5B900023E0FCA3E0FDEFD39DEE9C4068
:10332300091266948E5A8F5B8006755B00755A008E
:10333300AE5AAF5B741012664890006BE08E048F38
:1033430005FF1266388C5A8D5B74FFBC0009D39D50
:103353004005855B6180037561FE9000B3E0B401B5
:103363000280030233FBA20DB3B3500E900087E03B
:10337300A852B80005D39553500280719000C4E061
:103383008561F0A4FFAEF074648E048F05FF1266AE
:10339300388C5A8D5BE56B6016E56BC394FE500F5A
:1033A3009000DDE0B402089000CBE0640B60028083
:1033B30017AE5AAF5B74E7126648E56B8E048F0550
:1033C300FF1266388C5A8D5BAE5AAF5B9007BEE036
:1033D300FCA3E0FDEDD39FEC9E4005855B5F800B76
:1033E300A23BB340069007BFE0F55F800BA23BB35F
:1033F30040069007BFE0F55F800375610090008091
:10340300E07006756F0202305075BB1902384590A3
:103413000080E070030234B2E55ED39551400302AD
:1034230034B0900021E0FEA3E0FFE56512668C90C6
:103433000021EEF0A3EFF07E017F00E5BE126648A7
:10344300E5BD2FFF50010E8E5A8F5B9000EDE070AB
:1034530013740A12664874518E048F05FF1266387E
:103463008D658019AE5AAF5B740A1266488F048E5D
:10347300057E017F95CDCCCD1265368F65E565D38D
:1034830094644003756564900021E0FEA3E0FFE5CA
:10349300652FFF50010E900021EEF0A3EFF0900096
:1034A30084E0048E048F05FF1266388D65800375F2
:1034B30065329000D0E07006756F0302305075BB23
:1034C300130238459000D0E0604A7E017F00E5BEDC
:1034D300126648E5BD2FFF50010E8E5A8F5B7404B0
:1034E3001200398F669000D2E08566F0A4FDACF03F
:1034F3007464FF1266388D669000D1E08566F0A48F
:10350300FFAEF074FF8E048F05FF126638ED900056
:103513006AF0800375660090007EE07006756F04A4
:1035230002305075BB1702384590007EE0B40102AB
:1035330080030235C07E017F00E5BE126648E5BD0B
:103543002FFF50010E8E5A8F5B9007CBE0601990CE
:1035530007CBE014905FA812008CE493FC740193F2
:10356300FDEDC39FEC9E400280069007CBE014F074
:103573009007CBE0C394B3501DAE5AAF5B9007CB1B
:10358300E004905FA812008CE493FC740193FDEFB8
:10359300C39DEE9C400280069007CBE004F09007A9
:1035A300CBE0FE9000A4E08E0088F0A4FFAEF074A0
:1035B300648E048F05FF1266388D6780037567007C
:1035C30090007FE07006756F0502305075BB1602E0
:1035D300384590007FE0B4010280030236697E0122
:1035E3007F00E5BE126648E5BD2FFF50010E8E5ADF
:1035F3008F5B9007CCE060199007CCE014906112C8
:1036030012008CE493FC740193FDEDC39FEC9E4088
:103613000280069007CCE014F09007CCE0C394B38B
:10362300501DAE5AAF5B9007CCE0049061121200BC
:103633008CE493FC740193FDEFC39DEE9C400280E8
:10364300069007CCE004F09007CCE0FE9000AAE0DF
:103653008E0088F0A4FFAEF074648E048F05FF1211
:1036630066388D68800375680075BB1F0238457E18
:10367300017F00E5BE126648E5BD2FFF50010E8EA7
:103683005A8F5B740912664874E68E048F05FF1225
:1036930066388D6A900086E07006756F07023050B9
:1036A30075BB15023845900086E070030237C47E6F
:1036B300017F00E5BE126648E5BD2FFF50010E8E67
:1036C3005A8F5B74041200398F69900086E0B4014D
:1036D300159000DAE08569F0A4FFAEF074071200DC
:1036E30039EF9007C3F0900086E0B402159000DA3A
:1036F300E08569F0A4FFAEF07407120039EF90077C
:10370300C2F0900086E0B4030280030237A7900062
:10371300C7E0701CE569C394195002D22DE569D343
:1037230094644002C22D9000A6E09007C6F0806327
:103733009000A6E070349000DAE08569F0A4FFAE53
:10374300F074FF8E048F05FF126638ED9007C6F004
:10375300AE52AF53741EBE0006D39F4002D22DE576
:1037630061D394E54002C22D8029E569C3940A50D0
:103773000DAE52AF53741EBE0004D39F500280029D
:10378300D22DE561D394E54002C22D9000A6E090CE
:1037930007C6F09007C6E0C394055006740590076A
:1037A300C6F0C23C900086E0B40414E569C39419E2
:1037B3005002D23CE569D394324002C23CC22D8010
:1037C300037569009000DDE07006756F08023050E4
:1037D30075BB14806D9000DDE060567E017F00E5CF
:1037E300BE126648E5BD2FFF50010E8E5A8F5BEF68
:1037F300D39421EE940E4005756BFF8015AE5AAF3E
:103803005B741012664874E38E048F05FF126638EA
:103813008D6BE56B75F00BA4FFAEF09000CBE08EE3
:10382300048F05FF1266389007C0ECF0A3EDF0801B
:1038330003756B00900081E0600575BB1A8003750A
:02384300BB18B0
:1039F10002305902328C0234120234C702352C02D1
:0B3A010035D50236720236A90237D814
:05384500056FD2EC222A
:09667A002582F5825002058322FD
:0F008C0025E050020583258250020583F582226C
:10661700EF2F500205832582F582E5833E2EF58311
:016627002250
:10668C00CFC39FFF50011E22C3EF9DFFEE9CFE2245
:08669C000806B60002180622F0
:0D665600A3E004F07006120049E004F022F9
:0E003900048007C3CE13CECF13CFD5E0F6223E
:10653600BC000FBE0008ED8FF084FFADF022E4FE34
:10654600FF22BE000DEF60FE54F0606F20E70302ED
:1065560065ECEAC0E0EBC0E078017A0075F001EE88
:1065660020E710EF25E0FFEE33FE0AC5F023C5F065
:1065760030E7F0EA5407F9096A7A007B00600108FF
:10658600C3EC9E40167004ED9F4010ED9FFDEC9EFF
:10659600FCE5F0CA4ACA03F5F08005E5F003F5F01C
:1065A600C3EE13FEEF13FFD9D77908CACBCAD8D0EA
:1065B600EAFEEBFFD0E0FBD0E0FA22EC8FF084FCA1
:1065C600ED54F045F0C48FF084FEEDC454F045F070
:1065D600C48FF084FDEEC4FE54F02DFFEE540F3C44
:1065E600FEADF07C0022790078008FF0EC7E08206A
:1065F600E70DC3CD33CD33C933C9C833C8DEF08404
:1066060049F9E5F08FF0BE00E6FD7C00E9FFE8FE03
:016616002261
:0E664800F88FF0A4FFE5F0CE88F0A42EFE221D
:10000300EF8DF0A4F9A8F0EF8CF0A428F8EE8DF0B2
:06001300A428FEE9FF2213
:10662800600D782B026632007830D8FED5E0F8226B
:10663800EEC0E07E00126536EFFDEEFCD0E0FE22F3
:0C666300EEC0E07E00126536D0E0FE22A2
:03001B0002001EC2
:0300530002005652
:03009B00020071EF
:0300000002668312
:0966830075817575D0000242809A
:0B666F00E5822FF582E5833EF58322D3
:0A0049000582D5820215831582227C
:10001E00C0E0C0F0C083C082C0D075D0001241ECE9
:0B002E00D0D0D082D083D0F0D0E032E0
:10005600C0E0C0F0C083C082C0D075D0001241EFAE
:10006600D0D0D082D083D0F0D0E032C0E0C0F0C093
:1000760083C082C0D075D00012420BD0D0D082D0BF
:0600860083D0F0D0E0324F
:00000001FF
